:020000040000fa
:080000000001040000000000f3
:020000040000fa
:0400080040020000b2
:020000040000fa
:04000c0040020000ae
:020000040000fa
:0400100040020000aa
:020000040000fa
:0400140040020000a6
:020000040000fa
:0400180040020000a2
:020000040000fa
:04001c00400200009e
:020000040000fa
:04002000400200009a
:020000040000fa
:040024004002000096
:020000040000fa
:040028004002000092
:020000040000fa
:04002c00400200008e
:020000040000fa
:04003000400200008a
:020000040000fa
:040034001c4a000062
:020000040000fa
:040038004002000082
:020000040000fa
:04003c00400200007e
:020000040000fa
:04004000400200007a
:020000040000fa
:04004400364800003a
:020000040000fa
:040048004002000072
:020000040000fa
:04004c00400200006e
:020000040000fa
:04005000004200006a
:020000040000fa
:040054004c2c000030
:020000040000fa
:04005800482c000030
:020000040000fa
:04005c00400200005e
:020000040000fa
:04006000400200005a
:020000040000fa
:040064004002000056
:020000040000fa
:040068004002000052
:020000040000fa
:04006c00400200004e
:020000040000fa
:04007000400200004a
:020000040000fa
:040074004002000046
:020000040000fa
:040078004002000042
:020000040000fa
:04007c00400200003e
:020000040000fa
:04008000400200003a
:020000040000fa
:040084004002000036
:020000040000fa
:040088004002000032
:020000040000fa
:04008c00400200002e
:020000040000fa
:04009000400200002a
:020000040000fa
:040094004002000026
:020000040000fa
:040098004002000022
:020000040000fa
:04009c00400200001e
:020000040000fa
:0400a000a82c000088
:020000040000fa
:0400a400a42c000088
:020000040000fa
:0400a8004002000012
:020000040000fa
:0400ac00400200000e
:020000040000fa
:0400b000400200000a
:020000040000fa
:0400b4004002000006
:020000040000fa
:0400b8004002000002
:020000040000fa
:0400bc0040020000fe
:020000040000fa
:0400c00040020000fa
:020000040000fa
:0400c40040020000f6
:020000040000fa
:0400c80040020000f2
:020000040000fa
:0400cc0040020000ee
:020000040000fa
:0400d00040020000ea
:020000040000fa
:0400d40040020000e6
:020000040000fa
:0400d80040020000e2
:020000040000fa
:0400dc0040020000de
:020000040000fa
:0400e00040020000da
:020000040000fa
:0400e40040020000d6
:020000040000fa
:0400e80040020000d2
:020000040000fa
:0400ec0040020000ce
:020000040000fa
:0400f00040020000ca
:020000040000fa
:0400f40040020000c6
:020000040000fa
:0400f80040020000c2
:020000040000fa
:0400fc0040020000be
:020000040000fa
:0401000040020000b9
:020000040000fa
:0401040040020000b5
:020000040000fa
:0401080040020000b1
:020000040000fa
:04010c0040020000ad
:020000040000fa
:040110003242000077
:020000040000fa
:0401140040020000a5
:020000040000fa
:0401180040020000a1
:020000040000fa
:04011c00400200009d
:020000040000fa
:040120004002000099
:020000040000fa
:040124004002000095
:020000040000fa
:040128004002000091
:020000040000fa
:04012c00400200008d
:020000040000fa
:040130004002000089
:020000040000fa
:040134004002000085
:020000040000fa
:040138004002000081
:020000040000fa
:04013c00400200007d
:020000040000fa
:040140004002000079
:020000040000fa
:040144004002000075
:020000040000fa
:040148004002000071
:020000040000fa
:04014c00400200006d
:020000040000fa
:040150004002000069
:020000040000fa
:040154004002000065
:020000040000fa
:040158004002000061
:020000040000fa
:04015c00400200005d
:020000040000fa
:040160004002000059
:020000040000fa
:040164004002000055
:020000040000fa
:040168004002000051
:020000040000fa
:04016c00400200004d
:020000040000fa
:04017000042d00005a
:020000040000fa
:04017400002d00005a
:020000040000fa
:040178004002000041
:020000040000fa
:04017c00400200003d
:020000040000fa
:040180004002000039
:020000040000fa
:040184004002000035
:020000040000fa
:04018800602d0000e6
:020000040000fa
:04018c005c2d0000e6
:020000040000fa
:040190004002000029
:020000040000fa
:040194004002000025
:020000040000fa
:040198004002000021
:020000040000fa
:04019c00400200001d
:020000040000fa
:0401a0004002000019
:020000040000fa
:0401a4004002000015
:020000040000fa
:0401a8004002000011
:020000040000fa
:0401ac00400200000d
:020000040000fa
:0401b0004002000009
:020000040000fa
:0401b4004002000005
:020000040000fa
:0401b8004002000001
:020000040000fa
:0401bc0040020000fd
:020000040000fa
:0401c00040020000f9
:020000040000fa
:0401c40040020000f5
:020000040000fa
:0401c80040020000f1
:020000040000fa
:0401cc0040020000ed
:020000040000fa
:0401d00040020000e9
:020000040000fa
:0401d40040020000e5
:020000040000fa
:0401d80040020000e1
:020000040000fa
:0401dc0040020000dd
:020000040000fa
:0401e00040020000d9
:020000040000fa
:0401e400bc2d00002e
:020000040000fa
:0401e800b82d00002e
:020000040000fa
:0401ec0040020000cd
:020000040000fa
:0401f000182e0000c5
:020000040000fa
:0401f400142e0000c5
:020000040000fa
:0401f80040020000c1
:020000040000fa
:0401fc0040020000bd
:020000040000fa
:100200004f3724000e7f24000e01880000000000fc
:10021000000020000000e000020032000001200089
:10022000200288000c0007006082230001002000eb
:100230000f000700000020000000e0000200320074
:100240000000020000000000ee310200000000008b
:100250000040da000000fe00804120000000e000c5
:1002600002003200002020009001880000000600fb
:10027000a1028800800078000000eb001a0037001f
:10028000e280400054a0b4009101ba00e280400036
:1002900054a0b4009102ba00e280400054a0b4001f
:1002a0000002eb00472bde00f507b200a601880034
:1002b000602ce10008003a000049eb000201e80070
:1002c000020039003420ec0002f0a0008301e900b4
:1002d000f9ff3e00040037006128e1000100320010
:1002e0000082eb000b00070011c3ba001101ba0035
:1002f0000604e00003003a000200e000e0ff3a00dc
:1003000000000600f607b200a6028800820078000e
:10031000f5ff370004d0a300e20f49001c003900ac
:10032000810278003549ba000201e8000200390074
:100330003420ec0002f0a0008301e9000f0032003d
:100340002549ba000201e800020039003420ec001f
:1003500002f0a0008301e900080032000400e00080
:100360000600320015c9ba000201e8000200390097
:100370003420ec0002f0a0008301e9008180e80055
:1003800054a0b4000300e000e2ff3a0000000600c1
:100390009102ba00055978008301e900f7ff3200a5
:1003a000c82ade00055978008301e900f3ff320016
:1003b0000400e000f1ff320011d9ba00eeff37006f
:1003c0005e3f0400000000006e3f040000000000db
:1003d000c03f0400000000007a3f0400000000005d
:1003e0001040040000000000744004000000000001
:1003f000c440040000000000e035040000000000dc
:10040000f235040000000000443604000000000043
:10041000fe350400000000008836040000000000e3
:1004200058370400000000000638040000000000f7
:10043000704a0400000000008e4904000000000023
:100440007244040000000000224404000000000088
:10045000f843040000000000c04404000000000055
:100460004c45040000000000ae4504000000000000
:10047000fc450400000000002e49040000000000bc
:100480000040da000000fe009803e20004003d0096
:100490009b43ab00020032009b03ab00feff320027
:1004a0000040da00feff37000a00fa00e20f5000b9
:1004b00020003e00901b8200e10f50000600320039
:1004c000603b2000253b2000033b2000e43a200055
:1004d0000000e00004003a00003a2000c539200086
:1004e000a33920008439200006002800140363008b
:1004f00003003a000608780000002800140a700083
:1005000013a8a30001003a0013a0a0000200780085
:10051000050037001388a300feff32003102fb0004
:10052000840a78000000e9000000e000f9ff3a00ca
:100530000800370033002000b3bf9f00c0bf9f00fa
:10054000d1bf9f00e2bf9f006a805700620b070087
:100550006fb99700020078000080fa0000000600e2
:10056000839f68000100e00002003d006000100071
:10057000e08018000300e00002003d00600111006f
:10058000e0811900050007004f00e00002003b0079
:1005900060001000e0801800000006006022b80033
:1005a000060220000000d0008180d2000482d20028
:1005b0008582d2000000a0000202520083825a000d
:1005c000030031000202420083824a000000a100c1
:1005d0000603e900f3ff3a0000000600c42a2400e5
:1005e0000300e00002003a00932b2400030278008d
:1005f000831f7800841f7800801f7800811f780097
:10060000821f7800a02b2400801f78002030240057
:1006100001000700340007000000fa00688157005d
:10062000cfb89700010107000080fa000000060023
:100630008001780002003700b15978000201e9001a
:100640000200e000fcff3a00000006008001780094
:1006500002003700815978000201e9000200e00041
:10066000fcff3a00000006000001e9000080eb00fa
:10067000e50f510004003e000201410083352400d3
:100680006300790081317900000006008000e900f4
:10069000e58f50000f003e0081804000823524002d
:1006a000e28078000100e00002003a001000200023
:1006b00011000700e18f4000080032000001eb004c
:1006c000e18f500006003200010001000001eb0044
:1006d000030037000081eb000100370001017800c2
:1006e000020078000000060010002000e7ff07006d
:1006f000100020000000070000047800020007003e
:100700000800780060ff0700000006000800fa00fb
:10071000889fbe008a9fbe000084fb00d1c6b30044
:10072000814f5000340036004b06200011000900b4
:100730000b84d80081057800720040004300dd0082
:1007400029ff2300008044006022b800060020003a
:1007500007fe23005001be004000be00e00c070071
:100760000002be000203be0084bf9f0095bf9f0031
:10077000a6bf9f00b7bf9f00aa002000110009007c
:100780008a85d80080057800e9854500c35ddd00d5
:100790008b8544003b02be002b03be000fb89700c0
:1007a0009fb897002fb99700bfb99700cc0c0700ee
:1007b0000002be000203be0084bf9f0095bf9f00e1
:1007c000a6bf9f00b7bf9f00110009000a84d80090
:1007d000010478004344dd00888444003902be00ef
:1007e0002903be000fb897009fb897002fb9970054
:1007f000bfb997001d003700ea4f500013003600c4
:10080000aa002000110009000a84d8000105780020
:10081000690440004344dd0029ff230008844400ac
:100820006022b8000600200007fe23003800be004a
:100830002801be00aa0c07004355dd008a8444004d
:100840003902be002903be00080037004344dd0022
:1008500020ff2300080440006022b80006002000aa
:1008600007fe23003800be002801be009c0c0700d4
:100870004f05be004f04be000080fa0000000600d5
:100880000800fa00889fbe008a9fbe00d1c6b30050
:100890000004e00023003d000040ea000004fb00eb
:1008a000814f50000a003400420620001100090068
:1008b0000204d800a9002000110009008900d80016
:1008c000e9004000c308dd002aff230021003700b3
:1008d000ea4f500010003400a2002000110009006f
:1008e0000204d80001017800690040004300dd00e7
:1008f00021ff2300008040004311dd008280400082
:100900003102be002103be005001be004000be0007
:10091000730c0700380037004344dd0020ff23003c
:10092000320037000004fb00814f500023003400e8
:1009300042062000110009000204d800a90020008e
:10094000110009008900d800e9004000c308dd005b
:100950002af42300810045003102be002103be00bd
:100960008b0920008a8545003b00be002b01be009c
:100970005b0c07000002be000203be0084bf9f00a4
:1009800095bf9f00a6bf9f00b7bf9f001100090041
:100990000904d800010478004344dd00080545003f
:1009a0003a02be002a03be000fb897009fb8970016
:1009b0002fb99700bfb99700d5ff3700ea4f500015
:1009c00008003400a2002000110009000204d80031
:1009d00001017800690040004300dd0021f423009c
:1009e000c4ff37004344dd0020f423000804400026
:1009f0003800be002801be004f05be004f04be00f7
:100a00000080fa0000000600d00190000281510031
:100a10004240a90003003400100178000149780029
:100a20000208e8000100780000000600cf03b000d3
:100a3000889fbe008a9fbe008c9fbe008e1f7800dc
:100a40000006780091a79f00a2af9f006000b80049
:100a50006011b800a0a79f00b1a79f00c2a79f0088
:100a6000d3a79f008006eb008d0937009fa0970059
:100a70008100e80091a79f0051c2b300814f500050
:100a800003003a001fa197000007eb001100370098
:100a9000bc0090000000fb000168a30007003200ca
:100aa0000d017800800078000c007800d6ff070068
:100ab0000000e00005003a00790937008c0078005a
:100ac00083090700e10f4000750932008d06e80038
:100ad0007309370002007800b2407800b3c2b30057
:100ae00083cf50001300320007003c00ebc15100df
:100af00083cf50000d003200e3c1410083cf50008e
:100b000012003a000d003700d3c2b30083cf50006b
:100b100004003200e3c1410083cf50000b003a00d3
:100b2000080037000e30a000eaff37000e00a000da
:100b3000e8ff37000e10a000e6ff37000eb0a0005f
:100b4000e4ff37000e20a000e2ff37000e18a300dc
:100b5000010032000e00a1000e38a3000100320097
:100b60000e20a1000101fb000203b100e90f5100ba
:100b70000e003e00800078000001eb0082b79f006d
:100b80006a11b9003100fb000003b100020140000e
:100b9000010078009101fb000303b100e98f5100cf
:100ba000f7ff360082b79f000a0037008001eb0094
:100bb00083b79f00a2c2b30082cf500005003a0065
:100bc0002faa9700c4027800a4af9f0085b79f00aa
:100bd0000000e800e1c2b30090cf100017003a0017
:100be0000ee0a000e4c05000d0cf1000030032009f
:100bf000800078008001eb0009003700afab970060
:100c000047047800a7af9f00f8af9f000000e800fe
:100c1000800078000d0037006a1ab9008401410095
:100c2000010078003101fb000203b100e90f51001f
:100c3000f9ff3600f3af9f00f5ff37000ec0a000ac
:100c40008004eb00f9af9f00f1ff370031407800de
:100c500091a79f0072c6b300824f5000320032004d
:100c600017003c0031c6b300814f5000c200320073
:100c70000e003c00fcc05000814f50003d0032008f
:100c800006003c000004e0000a09320081c0e900cf
:100c9000814f5000d6003a003200370081c5b300c2
:100ca000814f5000d2003a003900370051c6b300de
:100cb000814f50001e00320027003c001e0037000c
:100cc00002c7b300824f5000310032000a003c00de
:100cd00064415100824f500019003200f1c6b30048
:100ce000814f500027003200e6c05000814f500075
:100cf000bf003a001000370051c7b300814f5000c9
:100d0000c2003200e3c04000814f500004003200b6
:100d1000e5c05000814f5000b5003a002000370078
:100d2000807f9f001c003700807f9f0013003700ea
:100d3000807f9f000d003700807f9f00b500370047
:100d4000000120000e48a30001003200000028002e
:100d50000e077000bdff3700807f9f000ea0a0002f
:100d6000ac003700807f9f000e50a0000e80a000d6
:100d7000a8003700807f9f000e50a0000e90a000ba
:100d8000a4003700807f9f000e60a000a100370004
:100d9000807f9f000e50a0000e70a0009d003700c5
:100da000807f9f00afad97004b007800abaf9f00f6
:100db00090b79f000000e00002003a00421c2400af
:100dc00092b79f009fb097000000eb000100370032
:100dd0000000e800614178000204e000fcff3a00f6
:100de000a0b79f00ffa997000300e00005003200b4
:100df0002fb29700848f51000200310083027800e7
:100e0000a5b79f002fb097000004eb000fb3970029
:100e1000800f53000100360000045300680767008c
:100e20002d003a00110037003c0090000068a3003c
:100e3000070032000d017800010220000c0078004c
:100e4000f1fe07000000e00006003a00060037004f
:100e50008c007800000220009d080700e10f400090
:100e6000010032008d06e8000804e9000800e000f7
:100e7000edff3a000084eb008e037800f7af9f008f
:100e8000170037003c0090000068a3000900320002
:100e900008007800b000fb00000478000d01780025
:100ea0000c007800d8fe07000000e00008003a00bf
:100eb00010003700880078003100fb000104780042
:100ec0008c00780082080700e10f40000900320022
:100ed0008d06e800070037008e047800f9af9f0008
:100ee000080778001fb49700afb497003fb597008c
:100ef000cfb59700090078008004e9000000e00009
:100f0000e0ff3a0098b79f00a9b79f00bab79f00cb
:100f1000cbb79f000e0478007faf97000e00e00073
:100f20005f083200110037003c0090000068a30009
:100f3000070032000d017800010220000c0078004b
:100f4000b1fe07000000e00006003a00060037008e
:100f50008c007800000220005d080700e10f4000cf
:100f6000010032008d06e8000804e9000800e000f6
:100f7000edff3a004a083700afa897004104780017
:100f8000a1af9f00cfc4de00614db9000802be00d2
:100f90000a03be004822de004829dd000402710079
:100fa000847f9f000e48a300090032000404e00083
:100fb00007003200e14f420005003200947f9f009d
:100fc000a87f9f0023002000a3b79f0003003700e5
:100fd000987f9f0014002000a4b79f0085fb2f007e
:100fe0008f8242008502e80095b79f007dff3700a1
:100ff000807f9f0086fb2f000683470096b79f00e7
:1010000017002000a7b79f0076ff3700807f9f0062
:101010000e0cb3000070200000006700990532003c
:101020000ec8a3000200320068002000f8af9f0045
:101030000e48a300050032002fa897004005be000f
:101040004004be00a0af9f00060037002fa9970004
:101050004200be00a2af9f00cc0907000004be0002
:101060000205be006022b8006033b8000800be0070
:101070000a01be00170907000000e00002003d0061
:101080000bf0a2003e00b3000000eb00e09f9f00c9
:101090006022b8006033b8000800be000a01be003c
:1010a000700907000000e00033003200c4fb2f008d
:1010b0000f0242000800be000a01be00560a0700e7
:1010c0006f9897000000e9006302b900a2002000b9
:1010d000110009000202d800e09f9f000000e0001c
:1010e00002003d000000e900e09f9f006f9997001b
:1010f00092b79f000240ea00e1fd07000802be002f
:101100000a03be00760a07000002be000203be000a
:10111000a4a79f00b5a79f00c6a79f00d7a79f00c1
:101120006022b8000600200007ff2300e90807003e
:101130000000e00003003d009fb297000500e900b9
:101140000c0037006022b80006002000470224008f
:101150002fa09700bfa097004fa19700dfa1970095
:10116000e10807000000e000030035001fb397000e
:101170000600e800e09f9f00ef9b970097b79f0055
:101180000e88a30008003a000e98a300180332004e
:1011900007007800e40f400003003500ffa8970027
:1011a000810f50009d0235007fa997000200e000ea
:1011b000040032000e98a300020032000201e90090
:1011c000f2af9f00ffa99700f28f51000300360095
:1011d00020c1b300807f9f00020037006fda9700c4
:1011e000847f9f006022b8006033b8000800be0012
:1011f0000a01be001b0907000000e0006600320083
:101200008f7a9700e5d79f002fe3970005405300a2
:101210009bfd07000002be000203be000800be00e6
:101220000a01be00b50807000004be000205be00aa
:10123000a6090700f60907000002be000203be006f
:101240000800be000a01be009a0a07006022b8002a
:101250000600200007fe2300a30807000000e000ae
:10126000080035006022b8000600200007fe2300b9
:101270000800be000a01be00190807000004be00f5
:101280000205be000800be000a01be008f0907006b
:101290000002be006033b800e4a79f00f5a79f00de
:1012a00086af9f0097af9f00efd297008502fb00ab
:1012b00085a79f000500e8004300dd00c61c240050
:1012c000000243003400be002401be00b0af9f0006
:1012d000c1af9f00d2af9f00e3af9f006fa2970006
:1012e000ffa297000fab97009fab97000020e10093
:1012f00001a8e10002b0e10003b8e1000c003900f0
:101300000400200005002a009699290097fb23007d
:101310000800be000a01be00f10907000004be007b
:101320000205be009fb297000500e80019003700d3
:101330000fa397004332dd00c71c24000482430042
:101340003400be002401be006fa29700ffa29700e8
:101350000fab97009fab97000020e10001a8e100d0
:1013600002b0e10003b8e1000b0031006022b800d8
:1013700006002000470224000800be000a01be004b
:10138000d70907000004be000205be009fb2970007
:101390000500e900e09f9f0001a020008100670098
:1013a00000202000808f50003d003a007fab970066
:1013b000f40f53000200340047012000f7af9f00f4
:1013c0000800be000a01be00400907006011b80015
:1013d0000802be000a03be0094b79f00a5b79f0095
:1013e000b6b79f00c7b79f0009003700ffaa970054
:1013f0008502e900f5af9f00a40020000500200051
:101400006033b8000800be000a01be00ca0a070027
:101410000205be000004be00e00f5000e08f58003f
:10142000e00f5900e08f590009003200a4002000ad
:10143000050020006033b800c60a0700e00f500026
:10144000e08f5800e00f5900e08f5900e7ff3200ad
:101450001fb49700afb497003fb59700cfb5970082
:101460000f7897008000fb007fab9700810f53003f
:101470000b003d000640500001fd07000002be00c9
:101480000203be000800be000a01be001b080700e0
:101490000004be000205be00efdb9700877f9f00bf
:1014a0008fb09700658050007fa997000200500020
:1014b00080b79f000200e00002003a000eb8a300cf
:1014c000030032008fb197008301e90083b79f00ca
:1014d00063006700030032000fb297000402e900c6
:1014e00084b79f000e28a3004f0032003c009000fc
:1014f000610167000e18a3000e0032000068a3000f
:1015000006003200b10220000200e00001003200bb
:101510008180e8000d0178000c003700b002200047
:101520000200e000010032000080e8008c0078003a
:101530000d0037000200e000320032000068a30016
:10154000070032000d017800010220000c00780035
:101550002dfd07000000e00006003a0029003700da
:101560008c00780000022000d9060700e10f40003f
:10157000240032008d06e800220037003c00900075
:101580000068a3000f0032000d0178000103200065
:101590000c007800f4b79f0085bf9f00d6b79f006e
:1015a000e7b79f0018fd07007fb297008fba97003a
:1015b0005fb39700efb397000000e0000e003a0021
:1015c0000e0037008c00780000032000f4b79f0065
:1015d00085bf9f00d6b79f00e7b79f00bc060700f6
:1015e0007fb297008fba97005fb39700efb3970071
:1015f000e10f4000010032008d06e8008904e90097
:10160000030037000802be000a03be008fb4970033
:101610000900e000d9ff3c0089b79f000404be0028
:101620000605be00450037000e38a30020003a0032
:101630000800be000a01be0090b79f00a1b79f003e
:10164000b2b79f00c3b79f008fb497001100370057
:101650003c0090000068a300070032000d017800f4
:10166000010220000c007800e7fc07000000e00009
:1016700006003a00060037008c00780000022000c7
:1016800093060700e10f4000010032008d06e800dc
:101690008904e9000900e000edff3c0089b79f00e4
:1016a0001fb49700afb497003fb59700cfb5970030
:1016b0003c009000610167000e18a3000e0032008c
:1016c0000068a30006003200b10220000200e00022
:1016d000010032008180e8000d0178000c00370025
:1016e000b00220000200e000010032000080e800ab
:1016f0008c0078000d0037000200e0000f0032007f
:101700000068a300070032000d01780001022000ec
:101710000c007800bcfc07000000e00006003a0066
:10172000060037008c0078000002200068060700e1
:10173000e10f4000010032008d06e8000800be0005
:101740000a01be00610807000002be006033b80055
:1017500094b79f00a5b79f00b6b79f00c7b79f007b
:101760003c019000c01c24008f7a97008500fb008c
:101770000268a30011003200c308dd0081004000b0
:101780003102be002103be001fb09700afb097002a
:101790003fb19700cfb19700e70907000003b00001
:1017a0000d017800800078000c00780096fc07009e
:1017b0000000e0000f003a000f003700c308dd0012
:1017c000810040003102be002103be001fb097001f
:1017d000afb097003fb19700cfb19700d60907008f
:1017e0000003b0008c00780039060700e10f4000cc
:1017f000010032008d06e8000f7b97000600fb0019
:101800004300dd00c11c2400008040003002be0007
:101810002003be001fb09700afb097003fb1970004
:10182000cfb19700cb09070090b79f00a1b79f00e9
:10183000b2b79f00c3b79f00ffac97000900e0005c
:1018400002003a000eb8a300740032003c00900081
:101850000068a300070032000d017800e1022000bb
:101860000c00780068fc07000000e00006003a0069
:10187000060037008c007800e00220001406070004
:10188000e10f4000010032008d06e8000f7c970058
:10189000e8d79f001fb49700afb497003fb59700fb
:1018a000cfb597003c0037000e98a3000d00320022
:1018b000e00f5400e08f5c00e00f5d00e08f5d0002
:1018c00008003a0098b79f00a9b79f00bab79f00d9
:1018d000cbb79f008040eb00817f9f000004eb00ae
:1018e0004c0037003c019000c11c24000000fb00ac
:1018f0000268a3000f0032004300dd0000804000ba
:101900003002be002003be000800be000a01be0077
:10191000890907000003b0000d01780080007800fd
:101920000c00780038fc07000000e0000d003a00d1
:101930000d0037004300dd00008040003002be0093
:101940002003be000800be000a01be007a0907009d
:101950000003b0008c007800dd050700e10f4000b7
:10196000010032008d06e8000f7997000200fb00ad
:101970004300dd00c11c2400008040003002be0096
:101980002003be000800be000a01be007109070066
:101990000205be000004be008f7897000140e900f8
:1019a000807f9f000104e000bfff3a0098b79f00ce
:1019b000a9b79f00bab79f00cbb79f006fd497001d
:1019c0000804fb00ffaa97000884520011003700aa
:1019d0003c0090000068a300070032000d01780071
:1019e000010320000c00780007fc07000000e00065
:1019f00006003a00060037008c0078000003200043
:101a0000b3050700e10f4000010032008d06e80039
:101a10000804e9000800e000edff3a003c009000f7
:101a20000e58a300080032000068a3000300320033
:101a30000d01780051042000070037008c00780069
:101a4000500420000b0037000068a300070032009c
:101a50000d017800510620000c007800eafb070019
:101a60000000e00006003a00060037008c00780015
:101a70005006200096050700e10f400001003200eb
:101a80008d06e800ef9897003c0090000100e00010
:101a90000a003d008100ea00e19f9f000068a3006a
:101aa000030032000d017800d1022000070037004a
:101ab0008c007800d00220000b0037000068a300e3
:101ac000070032000d017800b10220000c00780000
:101ad000cdfb07000000e00006003a0006003700da
:101ae0008c007800b002200079050700e10f40006b
:101af000010032008d06e800bc0090006f9897004e
:101b00000168a3000b003200a200200011000900b0
:101b10000200d80001032000808040000d01780001
:101b20000c007800b8fb07000000e00009003a0054
:101b300009003700a2002000110009000200d800af
:101b40000003b0008c00780061050700e10f400041
:101b5000010032008d06e800bc0090006f989700ed
:101b60000168a3000a003200a20020001100090051
:101b70000200d8000103b0000d0178000c007800cd
:101b8000a1fb07000000e0000a003a000a0037004d
:101b9000a2002000110009000200d800000320006c
:101ba000010040008c00780049050700e10f40006b
:101bb000010032008d06e8000e38a300380532001f
:101bc0000fb397000600e0003505340006047800e6
:101bd0003c0090000068a300070032000d0178006f
:101be000010220000c00780087fb07000000e000e5
:101bf00006003a00060037008c0078000002200042
:101c000033050700e10f4000010032008d06e800b7
:101c10000804e900eeff3a00210537009fb3970062
:101c20000700e00004003d000780ea00ffa89700dd
:101c300080804000f1af9f000800be000a01be0096
:101c4000f106070090b79f00a1b79f00b2b79f00b1
:101c5000c3b79f00c51c24000042eb000800be0073
:101c60000a01be00b0af9f00c1af9f00d2af9f007e
:101c7000e3af9f000c0037003500be003501be0009
:101c80001fb49700afb497003fb59700cfb597004a
:101c90000040e10001c8e10002d0e10003d8e1000a
:101ca000030039000442e800f44f5200f2ff3a000a
:101cb0003fac9700cfac97005fad9700efad9700ba
:101cc0000400fb00ffa8970080805000f1af9f0048
:101cd000f88f500009003c00014078008bfa0700a3
:101ce0000002be000203be000800be000a01be00e2
:101cf0007b0507000004be000205be006fd89700f8
:101d0000dffa07000002be000203be00b4af9f006e
:101d1000c5af9f00d6af9f00e7af9f001fb09700f1
:101d2000afb097003fb19700cfb197000d07070004
:101d30000002be000203be000800be000a01be0091
:101d4000dc0707000002be000203be003fa89700a8
:101d5000cfa897005fa99700efa997006007070039
:101d6000a90607000802be000a03be0094b79f0040
:101d7000a5b79f00b6b79f00c7b79f000205be007a
:101d80000004be000b003700a40020000500200066
:101d90006033b8000800be000a01be0066080700f4
:101da0000205be000004be00ffaa97008502e900fc
:101db000f5af9f007fab97000600e00019003200ee
:101dc000a4002000050020006033b8000800be0019
:101dd0000a01be005f080700e00f5000e08f5800c6
:101de000e00f5900e08f5900e7ff32000d00370087
:101df000ffab9700f88f53000e003c0007407800bf
:101e000042fa07000002be000203be000800be0046
:101e10000a01be00320507000004be000205be0034
:101e2000040037001fb49700afb497003fb5970088
:101e3000cfb597006f98970090b79f00e90f5000bb
:101e400012003c006022b8006033b8000800be00f9
:101e50000a01be00030607000000e0002f00320068
:101e60000800be000a01be0067060700e00f500030
:101e7000e08f5800e00f5900e08f590027003a002a
:101e80009fb09700e18f5000240034000400200030
:101e900005002e00b6e02200170124002fa09700b5
:101ea000bfa097004fa19700dfa197008905070009
:101eb0000000e00003003d001fb1970073005100d7
:101ec000020037009fb1970072805100e09f9f0091
:101ed0004f7897006afa07000002be000203be00b6
:101ee000a4a79f00b5a79f00c6a79f00d7a79f00e4
:101ef0000800be000a01be00800507004206070078
:101f000090b79f00a1b79f00b2b79f00c3b79f00d3
:101f10006044b8006055b800110037000800be00ea
:101f20000a01be003806070090b79f00a1b79f00c6
:101f3000b2b79f00c3b79f008a0607000002be0029
:101f40000203be000800be000a01be0059070700d8
:101f50000004be000205be000000eb00e09f9f00f1
:101f6000451d240014c0b3000800be000a01be00d5
:101f7000e0a79f00f1a79f0082af9f0093af9f0053
:101f8000100037003504be003505be00b8af9f0015
:101f9000c9af9f00daaf9f00ebaf9f001fb0970063
:101fa000afb097003fb19700cfb197000800e100b4
:101fb0000988e1000a90e1000b98e1000300390074
:101fc0000442e800f44f5200eeff3a006fa497007d
:101fd000ffa497000fad97009fad9700847f9f00ef
:101fe0006f9897008fb09700008050007fa99700ee
:101ff000820050000400fb000080500080b79f006a
:102000000080200000006700e0a79f0002003a0067
:102010000200e000030032008fb197008301e90065
:1020200083b79f0063006700030032000fb2970080
:102030000402e90084b79f000e28a300500032007c
:10204000610167000e18a3000f0032003c009000f1
:102050000068a30006003200b10220000200e00088
:10206000010032008180e8000d0178000d0037008a
:10207000b00220000200e000010032000080e80011
:102080008c0078000e0037000200e00033003200c0
:102090003c0090000068a300070032000d017800aa
:1020a000010220000c00780057fa07000000e00051
:1020b00006003a00290037008c007800000220005a
:1020c00003040700e10f4000240032008d06e80001
:1020d000220037003c0090000068a3000f0032008f
:1020e0000d017800010320000c007800f4b79f0078
:1020f00085bf9f00d6b79f00e7b79f0042fa070051
:102100007fb297008fba97005fb39700efb3970045
:102110000000e0000e003a000e0037008c0078004e
:1021200000032000f4b79f0085bf9f00d6b79f0033
:10213000e7b79f00e60307007fb297008fba9700ca
:102140005fb39700efb39700e10f4000010032004a
:102150008d06e8008904e900030037000802be008c
:102160000a03be008fb497000900e000d9ff3c00cd
:1021700089b79f000404be000605be007a00370040
:102180000e38a30020003a000802be000a03be0079
:10219000b4af9f00c5af9f00d6af9f00e7af9f00d1
:1021a0008fb49700110037003c0090000068a30036
:1021b000070032000d017800010220000c007800b9
:1021c00011fa07000000e00006003a0006003700a0
:1021d0008c00780000022000bd030700e10f4000e2
:1021e000010032008d06e8008904e9000900e000e2
:1021f000edff3c0089b79f003fac9700cfac970044
:102200005fad9700efad9700610167000e18a30066
:102210000f0032003c0090000068a300060032006e
:10222000b10220000200e000010032008180e800dd
:102230000d0178000d003700b00220000200e00020
:10224000010032000080e8008c0078000e003700aa
:102250000200e0003d0032003c0090000068a30056
:10226000070032000d017800010220000c00780008
:10227000e5f907000000e00006003a003a003700e8
:102280008c0078000002200091030700e10f40005d
:10229000350032008d06e8002c0037003c0190002c
:1022a000c01c24008100fb000268a3001300320060
:1022b000c308dd00010040003002be002003be0064
:1022c0000800be000a01be001b070700a400200092
:1022d000050020006033b8001e070700010320003e
:1022e000808040000d0178000c007800c6f90700de
:1022f0000000e00013003a0025003700c308dd00ad
:10230000010040003002be002003be000800be00f5
:102310000a01be0008070700a400200005002000f5
:102320006033b8000b0707000203200000014100e2
:102330008c0078000200780065030700e10f400080
:10234000130032008d06e800110037000802be00bd
:102350000a03be00b4af9f00c5af9f00d6af9f0079
:10236000e7af9f00060037000800be000a01be006c
:10237000b0af9f00c1af9f00d2af9f00e3af9f00ff
:102380001fb49700afb497003fb59700cfb5970043
:102390000f7897008040e900817f9f000004e000f3
:1023a000beff3a003fac9700cfac97005fad9700ff
:1023b000efad9700130037003c0090000068a300c9
:1023c000070032000d017800010320000c007800a6
:1023d0008df907000000e00006003a000600370013
:1023e0008c0078000003200039030700e10f400053
:1023f000010032008d06e8006f9897000000e900a8
:10240000e09f9f006f9897000000e000eaff3c000b
:10241000ffa89700f28f50000300340020c1b300e2
:10242000807f9f00020037006fd99700827f9f0056
:102430000f7897008000fb00ffa997008180510072
:10244000f1af9f000004e00003003a006fa2970084
:102450000400e000100032003c0090000068a3007f
:10246000070032000d017800e10220000c00780026
:1024700065f907000000e00006003a00060037009a
:102480008c007800e002200011030700e10f4000fb
:10249000010032008d06e8000f789700f8f8070079
:1024a0000002be000203be000800be000a01be001a
:1024b0008b050700d40407000205be000004be001f
:1024c00090b79f00a1b79f00b2b79f00c3b79f000e
:1024d000350037003c019000c11c24000000fb00c7
:1024e0000268a300130032004300dd0000804000ba
:1024f0003002be002003be000800be000a01be007c
:102500008d060700a4002000050020006033b800fd
:10251000900607000003b0000d01780080007800ed
:102520000c00780038f907000000e00011003a00c4
:10253000110037004300dd00008040003002be0083
:102540002003be000800be000a01be007a06070094
:10255000a4002000050020006033b8007d060700bd
:102560000003b0008c007800d9020700e10f4000a2
:10257000010032008d06e8008f7897000100fb0013
:102580004300dd00c11c2400008040003002be007a
:102590002003be000800be000a01be006d06070051
:1025a0000205be000004be008f7897000140e900dc
:1025b000807f9f000104e000c6ff3a0098b79f00ab
:1025c000a9b79f00bab79f00cbb79f007fac970019
:1025d000110037003c0090000068a30007003200a3
:1025e0000d017800010320000c00780006f90700b7
:1025f0000000e00006003a00060037008c0078007a
:1026000000032000b2020700e10f40000100320089
:102610008d06e8000804e9000800e000edff3a003c
:102620000e38a3009e0232008fb297000500e00032
:102630009b023400050478003c0090000068a30071
:10264000070032000d017800010220000c00780024
:10265000edf807000000e00006003a000600370031
:102660008c0078000002200099020700e10f400072
:10267000010032008d06e8000804e900eeff3a0090
:10268000870237000e007800000cb20032003a00da
:102690000e00e00005003d002fa897004005be0099
:1026a0004004be00a0af9f00120037000e48a300f8
:1026b0000b0032002fa997004200be00a2af9f007e
:1026c0000002be004fabde008603780094b79f0087
:1026d000a5b79f00b6b79f00c7b79f000900370096
:1026e000afaa970045007800a5af9f006104b9002c
:1026f000614db90098b79f00a9b79f00bab79f0076
:10270000cbb79f001fb09700afb097003fb19700c5
:10271000cfb19700e00f5000e08f5800e00f590054
:10272000e08f590027003d003e00b3006000b80074
:102730006011b8001fb29700afb297003fb3970087
:10274000cfb3970004025000858258000603590059
:1027500087835900170037000e00e00009003d0094
:102760002fa897004005be004004be00a0af9f0008
:1027700098b79f00a9b79f00bab79f00cbb79f003b
:10278000100037000e48a300050032002fac970060
:102790004802be006033b800a8af9f0005003700b4
:1027a000afac970049007800a9af9f006102b80064
:1027b0006033b80094b79f00a5b79f00b6b79f00dd
:1027c000c7b79f00ffaa97000500e0000d003a0080
:1027d00016002000f6af9f001fb49700afb497001b
:1027e0003fb59700cfb59700e00f5400e08f5c0035
:1027f000e00f5d00e08f5d00020032008004eb001e
:10280000f9af9f000e0578000a0cb200baaf9f0026
:1028100000042000800f55003400320003003c000b
:102820000a00e000080032004800370000082000dd
:10283000bfad9700808f550014003200000c2000bf
:10284000808f550041003a00451d240014c0b3009c
:102850003500be003501be001fb49700afb497002d
:102860003fb59700cfb597000040e10001c8e100f7
:1028700002d0e10003d8e100330039000442e8004f
:10288000f44f5200f2ff3a002f00370014c0b3009b
:1028900000012000010020006011b8001fb4970063
:1028a000afb497003fb59700cfb597000040e10067
:1028b00001c8e10002d0e10003d8e10022003900a4
:1028c000490020000000d0008180d2000281d200a7
:1028d0008381d2008904e900faff3a000442e8004b
:1028e000f04f5200edff3a001700370014c0b3005c
:1028f00080002000010020006011b8001fb4970084
:10290000afb497003fb59700cfb597000040e10006
:1029100001c8e10002d0e10003d8e1000a0039005b
:10292000390020000000d0008180d2000281d20056
:102930008381d2008904e900faff3a000442e800ea
:10294000f54f5200edff3a00847f9f000f7d970006
:102950000a00fb00ffad97008b0f500002003d0006
:102960008b7f9f0004003700ffa89700808f5000e6
:1029700001003d00f0af9f000fb197000200e000a2
:102980000400320063006700020032000201e90027
:1029900082b79f000ee8a300090032008fb19700b4
:1029a0007faa9700848f5100030034008481510076
:1029b00083b79f00020037008002eb0085b79f00bd
:1029c000418c20008100670000842000808f50002f
:1029d00006003a000fb397000600e0001000320036
:1029e0000603e90086b79f000d003700018c200028
:1029f0008100670000882000808f500008003a00a6
:102a00008fb39700e28f5300030034008783e900ff
:102a100087b79f00020037000004eb0088b79f00d3
:102a20008f7c97000900fb000005eb00eaa79f00e0
:102a30008fb59700808f550002003400008055004c
:102a4000e0a79f000e28a30060003200610167002c
:102a50000e18a3000d0032003c0090000068a30097
:102a600005003200b10220000200e0003000320018
:102a70008180e8002e003700b00220000200e00054
:102a8000350032000080e800330037000200e0002b
:102a9000090032003c0090000068a30003003200ef
:102aa0000d01780001022000220037008c00780020
:102ab0000002200029003700018c200081006700ff
:102ac00000882000808f500028003a003c009000d1
:102ad0000068a300070032000d0178000103200008
:102ae0000c007800c8f707000000e00006003a007c
:102af000060037008c0078000003200074010700f6
:102b0000e10f4000010032008d06e8003c0090001b
:102b10000e0178000202b2000068a3000a00320031
:102b2000810720000200e000010032008105200042
:102b30000d0178000c007800b3f707000000e000fa
:102b400009003a0009003700800720000200e00079
:102b500001003200800520008c0078005c01070035
:102b6000e10f4000010032008d06e8006fa09700e1
:102b70000000e0008b003200000478003c00900070
:102b80000068a300070032000d0178000103200057
:102b90000c0078009cf707000000e00006003a00f7
:102ba000060037008c007800000320004801070071
:102bb000e10f4000010032008d06e8000804e90042
:102bc000eeff3a00e8a79f0076003700efa09700dd
:102bd0000100e000160032000e38a30014003a0095
:102be000010478003c0090000068a3000700320058
:102bf0000d017800010220000c00780082f7070028
:102c00000000e00006003a00060037008c00780063
:102c1000000220002e010700e10f400001003200f9
:102c20008d06e8000804e900eeff3a00e8a79f00df
:102c3000610167000e18a3000f0032003c009000f5
:102c40000068a30006003200b10220000200e0008c
:102c5000010032008180e8000d0178000d0037008e
:102c6000b00220000200e000010032000080e80015
:102c70008c0078000e0037000200e00010003200e7
:102c80003c0090000068a300070032000d017800ae
:102c9000010220000c0078005bf707000000e00054
:102ca00006003a00060037008c0078000002200081
:102cb00007010700e10f4000010032008d06e80027
:102cc000008c20000000670001842000810f50006c
:102cd00009003a003c0090000068a30003003200a5
:102ce0000d01780001032000200037008c007800df
:102cf000000320002700370001882000810f5000ca
:102d000028003a003c0090000068a3000700320051
:102d10000d017800010320000c0078003af707004d
:102d20000000e00006003a00060037008c00780042
:102d300000032000e6000700e10f40000100320020
:102d40008d06e8003c0090000e0178000202b200ff
:102d50000068a3000a003200810720000200e000a2
:102d600001003200810520000d0178000c00780080
:102d700025f707000000e00009003a0009003700cd
:102d8000800720000200e0000100320080052000e2
:102d90008c007800ce000700e10f400001003200f7
:102da0008d06e8007fa997000200e900c201dd005e
:102db00083a79f006301b90002027800f49f9f007f
:102dc0004300dd00c11c24008100400081b79f004a
:102dd00098003700ffaa97008502e900f5af9f0031
:102de000000420003fab9700800f530068003200c2
:102df00003003c000600e0000800320073003700ca
:102e000000082000bfab9700808f53004c003200b9
:102e1000000c2000808f53006c003a000e00e00090
:102e20001e003d000fb097003004be002005be001c
:102e30000802be000a03be001fb09700afb09700a3
:102e40003fb19700cfb197003b040700807f9f0000
:102e50000000fb00cf80de006109b9000802be005f
:102e60000a03be009d0407001fb29700afb297008f
:102e70003fb39700cfb397000002520081825a00ff
:102e800002035b0083835b0094b79f00a5b79f009c
:102e9000b6b79f00c7b79f00250037000e48a300b4
:102ea0001a0032001fb29700afb297000fb397001d
:102eb0003604be002605be000801be000400be00a8
:102ec000f4b79f0085bf9f00b4f50700807f9f0087
:102ed0000000fb00cf80de000801be007703070082
:102ee0007fb297008fba97000000520081805a008d
:102ef0000004be006055b80098b79f00a9b79f00b6
:102f0000bab79f00cbb79f00090037008fb4970076
:102f1000190178001fb59700110009000285d8003b
:102f2000a2002000110009000280d800817f9f00cc
:102f30008f7d97000b43b0008b7f9f0023003700ed
:102f4000301b24000e58a30001003200201a240078
:102f50001fb29700afb297003fb39700cfb397006f
:102f60008fa097008100e900050033008703d1009e
:102f70000683d3008582d3000482d300f9ff370093
:102f80006f02620060427a00847f9f000f0037006a
:102f90001fb09700afb097003fb19700cfb1970037
:102fa0007f9a97000402e900050033008301d100f5
:102fb0000281d3008180d3000080d300f9ff370065
:102fc000674060000043b000807f9f00bc0090001d
:102fd0008f7a97000500fb000168a300070032000c
:102fe0000d017800800078000c00780086f607005c
:102ff0000000e00005003a00050037008c00780072
:1030000033000700e10f4000010032008d06e800a8
:103010000fa397006403530086a79f00ff9b9700b0
:10302000e3835300f79f9f000fb497006804540098
:1030300088b79f00ffac97000900e00065ff3a00e9
:103040000e38a300160032006fa597000a00e000ba
:10305000130034000a0478003c0090000068a300cc
:10306000070032000d017800010220000c007800fa
:1030700065f607000000e00006003a000600370091
:103080008c0078000002200011000700e10f4000d2
:10309000010032008d06e8000804e900eeff3a0066
:1030a0009fa597001b407800807f9f000004e000f0
:1030b0006ef63a000d0078004f0778004f06be000c
:1030c0004f05be004f04be00cf03b1000000060054
:1030d000889fbe0001047800b80090008084eb0057
:1030e0000118a3003a003200180190000198a300d3
:1030f00002003a000200e00035003a000190a00012
:103100003104980080047800f90fb2000200e0005a
:1031100002003a0028009000000c7800ea8f54006a
:1031200005003a000178a30003003a008800780007
:10313000d0002000e6ff070018009000d8009000a3
:10314000810f50000b0032000000e80010049800ce
:103150001800780009487800000ce80011c0b3009e
:10316000c036240001487800ea8f540018003a0065
:103170000500370088007800094078001700070034
:103180008004780012003700380090000088a30007
:103190000f00320018019000a80090004800900035
:1031a000c1f4070098009000810f50000400320025
:1031b000380090000003b300300498008084eb00d6
:1031c0000000eb001004980028009000000c78002c
:1031d000090078004f04be00000006000200fa005b
:1031e000889fbe00a0ff9f00010478003800900077
:1031f0000068a30033003a00e200600005003a00d6
:103200000003b30030049800110498000080eb0024
:103210002e003700d80490000900e00006003a00b4
:1032200012002000e6805700480090009ef407003e
:103230001904980023003700a80090000100e00066
:1032400008003a00f136240021049800010c7800af
:103250002100200051049800110498000030a000c3
:103260003004980018019000a800900048009000d9
:103270008df40700280090008080eb001104980076
:10328000aff8970001487800000ce8002ff897008d
:10329000ea4f50000b003a00380090000088a3006d
:1032a0000800320018019000a8009000480090002b
:1032b0007df407000000eb0010049800a8009000c7
:1032c000010c7800aff897000100fb004f04be002e
:1032d0000080fa000000060000c0da0000000600ce
:1032e0002800fa00889fbe008a9fbe008c9fbe0007
:1032f00007067800878669000c003b00030478000d
:103300008704780008f0a10009f0a100840f5000a4
:10331000858f5800860f5900890f5c000300330029
:103320000cf0a20001003a000cf0a100fe00070022
:103330006400e1005f003200780147006408e100aa
:10334000610032006c014700748557003200be00f6
:103350001201be003a04be001a05be001e03900012
:10336000be0a90008503530006003d000004fd00e6
:103370008104fd000205fd008305fd008703ea00ce
:10338000050378000df8a300040032006004140067
:10339000e0841c0060051d00e0851d006022b8006f
:1033a0007d0320000d38e1008006eb000b003900a2
:1033b0004433dd00f300b2008301730039003700ad
:1033c000848272000d027800e10664008b85d100d2
:1033d0000a85d3008984d3000884d3008703e900d9
:1033e000f7ff3b0008004000898048000a014900bf
:1033f0008b81490004003b0060001000e080180051
:1034000060011900e08119000358a300090032008f
:103410008d82720084827200610260008301d1009b
:103420000281d3008180d3000080d3000603e8002e
:103430001b0037000348a30017003a000600e00015
:10344000170034000603e9000d00a3000000480047
:103450008180480002014900838149000348a3009c
:103460000f003a000600e000090034000603e900fe
:10347000000040008180480002014900838149002a
:1034800001003a000003eb000348a300f5ff3200ff
:103490006022b800020037008482720061826600f8
:1034a0007500070003f0a1000cf0a70003f0a000d6
:1034b000b1003700640147006408e10002003a00ef
:1034c0000df8a300a9003a003200be001201be00b0
:1034d000a90037008f1fd100290307008f87e9005b
:1034e0000000e00000000600809feb0024030700be
:1034f0008f87e9000000e000000006002800fa00c5
:10350000889fbe008a9fbe008c9fbe0003866b0012
:10351000850007006400e100440032006408e10017
:103520004a0032006100e100460032006108e1001b
:1035300049003200ec0647006000b8003d02be00c2
:103540003d03be00f48657006011b8003d04be0084
:103550003d05be007d0320000b0037000000a000e9
:103560008d06e900130032000402420085824a0001
:1035700006034b0087834b00000040008180480019
:1035800002014900838149000802520089825a00e1
:103590000a035b008b835b00f0ff3b0008024200e4
:1035a00089824a000a034b008b834b008d06e90099
:1035b000edff3a008482720086827200f707b20043
:1035c0008782720001003200150020001e04900066
:1035d0003e0b900006035400e63fb0000368a300d2
:1035e000070032000000a7000500a0008301d10001
:1035f0000281d3008180d3000080d3000603e8005d
:103600008301d1000281d3008180d3000080d300e8
:103610000002eb000482d2001700070003f0a100b3
:103620000cf0a70003f0a00053003700640247002d
:103630006408e1004d0032003400be003401be00d9
:10364000f6ff37006108e100480032006011b80061
:103650006000b800f1ff370003ff270002002000e0
:10366000fbff3700801feb00c50207008f87e900d2
:103670000000e000000006001800200057002000b5
:10368000080453000d003d000600200097fc2f00a9
:103690000740e1001e003400848272006102600075
:1036a0008301d1000281d3008180d3000080d30048
:1036b0000804e800f8ff3a004700200061046000b9
:1036c00005047400040464000d0032006100400031
:1036d000e080480060014900e081490003b8a5008e
:1036e000070032000603e8006538e10004003a00f4
:1036f0008301d1000281d3008180d3000080d300f8
:10370000f87f20000830e10003003500080378004e
:103710006000b8006011b8004433dd00f300b2006f
:103720008301730000000600680447000294be0095
:103730000094be00fc0447008694be008494be0042
:1037400009007800d702070008007800d5020700ba
:1037500099007800814f70000b003b000800be000c
:10376000b00207004f00b10003003700f3ff27004d
:10377000f2ff2f006110b9004f06be004f05be00da
:103780004f04be000080fa000000060081037800ac
:10379000be0007000001be006000b8000478a3006e
:1037a00013003a006220e10015003e000d003900d0
:1037b0008301d1000281d3008180d3008301d10035
:1037c0000281d3008180d3008301d1000281d30024
:1037d0008180d3000538b000c42add00f300b200b8
:1037e0008381720007f0a70003f0a000000006002c
:1037f000f3ff2700f2ff2f006110b900fbff370035
:1038000003ff2700f7ff37001400fa00889fbe006f
:103810008a9fbe008c9fbe000004be000205be0051
:10382000680047000a90be000890be009d02070095
:103830000070a7000bf0a1000bf8a30020003a00d5
:103840009e0990000e099000fe0090006e0090000e
:103850009e0290003443200084825200c6ff320052
:103860000a003c00b4fc2f000428e10014003400de
:103870008301d1000281d3008180d3000080d30076
:103880008502e800faff3a00bbff3700b4002000d1
:103890000428e10007003c0000004000818048004f
:1038a00002014900838149008502e900faff3a00dc
:1038b000b1ff37000300280002002000010037009c
:1038c0006011b8006000b800abff37001400fa00c8
:1038d000889fbe008a9fbe008c9fbe000004be0071
:1038e0000205be00680047000a90be000890be00b6
:1038f0006c0207000070a7000bf0a1000bf8a300fa
:1039000016003a009e029000304320008082520050
:10391000b0fe2f000028e1000d003c00b0fc2f009d
:103920000028e1000d0034001e0990008e08900070
:103930007e0090000501b0000201d1008180d3001b
:103940000080d3008502e800fbff3a008aff3700c1
:10395000010028000000200087ff37006000b80049
:1039600085ff3700889fbe0000827000040271004e
:10397000048271002400320036432000c50020007c
:103980008383cf000a0039000541b1008283cf0054
:10399000070039000541b1008183cf0004003900e0
:1039a0000541b1008083cf00010039000541b1001d
:1039b00085c353006022b800120032000a003b00a9
:1039c00084827200610260008301d1000281d30011
:1039d0008180d3000080d3000603e8008743e8001d
:1039e000f7ff3a00070037000000400081804800e0
:1039f00002014900838149000603e9008743e90089
:103a0000f9ff3a001cff07004f04be00000006004b
:103a10006011b800d3ff37001400fa00889fbe0081
:103a20008a9fbe008c9fbe00040678000004be0082
:103a30000205be00680047000a90be000890be0064
:103a4000180207006200e1000800be000a01be0083
:103a5000040020000b003a001e029000e43fb10079
:103a60006e009000fe0090000e0990009e099000ec
:103a7000f300b20005fe2300858171000bf0a70062
:103a800003f0a000040e78003bff3700c70ade00f9
:103a9000f107b200f50fb20008003200e1cf42009a
:103aa000020032000170a00024000500810f7000a8
:103ab000010032000408050044000500810f700079
:103ac00002003a00140005008502e90000004000f1
:103ad00081c04800fcff3b000170a00024000500ed
:103ae0002800fa00889fbe008a9fbe008c9fbe00ff
:103af00003866b000cff07000028a30064003a0057
:103b00000128a30067003a000008a30062003a0001
:103b10000108a30065003a001e009000be08900056
:103b200081064000ed3fb100f4805700ee019000a7
:103b3000111ab8008e099000311bb8009e09900040
:103b4000311cb800511db800f4855700460007002d
:103b5000fe0190003a0007008b85e8003e00070058
:103b60008e09900040000700ee019000340007002d
:103b70008b85e800380007008e09900040000700a0
:103b80009e0990001b18b800890440000a8548006f
:103b9000fe019000340007008b85e8003800070024
:103ba000ee019000300007008e0990001b18b8004d
:103bb000890440000a8548000a98a30008003a00da
:103bc0000402420085824a0006034b0087834b00b3
:103bd00008044c0089844c000a054d008d06e9005c
:103be00084827200850273004c3add008502720007
:103bf0000100320015002000443ade001400b2003b
:103c00004538de00cb45dd000b007000c540de000e
:103c1000cb4ddd008b8070004549de00cb55dd00cb
:103c20000b017100c551de000d03780092fe070004
:103c300003f0a1000cf0a70003f0a000cefe3700b7
:103c40001b18b8008502400006834800e0834b0043
:103c500060044c00070037001b18b8000603400042
:103c600087834800faff37001b18b800870340001d
:103c700008844800e0844c0060054d000000060008
:103c80001b18b8000804400089844800faff370078
:103c90000108a300b5fe3a005800be005801be005e
:103ca000e3ff37000008a300b0fe3a0009047800e3
:103cb000f9ff370007f0a20089fd3700020ab900ba
:103cc000001bb9000200b8008100420081004300df
:103cd00000000600889fbe008a9fbe00300442009c
:103ce000b0844a0030054b0090854b006000b10065
:103cf0000898be000a90be000440e10005c8e1003b
:103d000006d0e10007d8e100020031006800400061
:103d10001008e8004f05be004f04be00000006007a
:103d2000889fbe008a9fbe003004be002005be00f2
:103d30000418540005985c0006185d0007985d00a3
:103d4000110020000440e10005c8e10006d0e100b8
:103d500007d8e100010039008000eb001088100056
:103d60004f05be004f04be00000006001200fa001e
:103d7000889fbe008a9fbe008c9fbe00e0b79f0058
:103d8000f1b79f0082bf9f0093bf9f000605be0052
:103d90000404be000000eb00d0b79f00c0b79f0036
:103da000b0b79f00a0b79f0090b79f000006eb0040
:103db0005fb19700cfb09700820141003fb09700fc
:103dc0000200e00004003d00370007007e8057003d
:103dd000c0ff070003003700330007007e80570054
:103de000cfff0700dfb697000d00e0000c003500a4
:103df0006fb29700ffb297000fbb97009fbb970071
:103e000010002000010020006011b80000027200c4
:103e10008182720002037300838373001b0007001a
:103e20000c06e80001042000810f5600e0ff3a0074
:103e30000d00e00004003d000802be000a03be00c1
:103e40007e805700a3ff07005fa897000000e000f6
:103e500005003a001fb29700afb297003fb397003a
:103e6000cfb39700090007006fb09700ffb097002d
:103e70000fb997009fb997004f06be004f05be00cf
:103e80004f04be000080fa00000006000100070099
:103e900000000600a4b79f00b5b79f00c6b79f00fb
:103ea000d7b79f00000006004f09de008281710035
:103eb000b3b79f004f01de00818040008280700018
:103ec000a1b79f008fb097004f09de0000004000af
:103ed0000200700090b79f007fa897004f01de009e
:103ee000818040008280700081b79f000d00070034
:103ef0004f3ade000000400004007000f0af9f0069
:103f0000080007000402420085824a0006034b00b5
:103f100087834b00dfff07000802be000a03be00d4
:103f2000000006002fb29700bfb297004fb3970072
:103f3000dfb3970000000600881f780018002000fb
:103f4000881f780089ff07008f87e9004f047800f9
:103f500000000600801feb0084ff07008f87e90048
:103f600000000600889fbe008a9fbe00e00f500040
:103f7000e08f5800e00f5900e08f59000c003d0021
:103f80006044b8006055b8000000540081805c00b7
:103f900002015d0083815d0018002000150007000c
:103fa00008003d00180007000004eb000500370082
:103fb0000004eb000f00070002003d0012000700a4
:103fc00018002000dcff07000800e00006003200b7
:103fd0006022b8006033b8000000520081805a00af
:103fe00002015b0083815b004f05be004f04be00f1
:103ff00000000600e00f5200e08f5a00e00f5b0067
:10400000e08f5b00000006006044b8006055b80017
:104010000402540085825c0006035d0087835d0016
:1040200000000600889fbe008a9fbe008c1f78009b
:10403000e00f5000e08f5800e00f5900e08f59006a
:104040000d003d006044b8006055b8000000540009
:1040500081805c0002015d0083815d001c00200006
:104060000820e10009a8e1000ab0e1000bb8e10076
:104070000d003d00080037000006eb00e00f520085
:10408000e08f5a00e00f5b00e08f5b0006003d0010
:104090006044b8006055b8000402540085825c009a
:1040a00006035d0087835d00aaff07000c00e000a7
:1040b000060032006022b8006033b80000005200f1
:1040c00081805a0002015b0083815b004f0678000b
:1040d0004f05be004f04be0000000600889fbe00d2
:1040e0008a9fbe008c1f78000006eb00e00f500096
:1040f000e08f5800e00f5900e08f590007003d00a5
:104100006044b8006055b8000000540081805c0035
:1041100002015d0083815d001c002000e00f520061
:10412000e08f5a00e00f5b00e08f5b0007003d006e
:104130006044b8006055b8000402540085825c00f9
:1041400006035d0087835d000c00a2007c00070071
:104150000c00e000060032006022b8006033b800b6
:104160000000520081805a0002015b0083815b00e5
:104170004f0678004f05be004f04be000000060049
:10418000889fbe008a9fbe008c9fbe000404be00b4
:104190000605be00809fbe00829fbe002f00070064
:1041a000040678000800be000a01be002b000700cc
:1041b000840678004f03be004f02be008d4f76008c
:1041c0007fb0970013003300f0ff2f008b8f6b0040
:1041d00006003b000d0666000c00a7000a00370031
:1041e00007f0a600100020000a003700880f5200d8
:1041f000898f5a008a0f5b008b8f5b0003003900a8
:104200001000200001003e000000200007f0a70081
:104210000000ea004f06be004f05be004f04be007e
:1042200000000600e48240001078a300070032007e
:10423000640240001178a3003400be001401be00e7
:10424000040032000330a700000006003500be0065
:104250001501be000330a0000000060005ff270086
:1042600005826100070032000428e10001003200ed
:10427000240005000600070001003a004400050084
:104280000408050002000700f9ff3a0014000500c9
:104290006f826100810270008502710085027200e8
:1042a00000000600800078005002be005003be00ef
:1042b0004439de00f700b200f37f20000301610003
:1042c000090032000218e10016003a008501720070
:1042d00083017300838173000008200015003a00f9
:1042e0004000200013003700850172008301730035
:1042f0008381730005003a0004a8be0006a8be0032
:10430000100020000b0037000201e9000402420007
:1043100085824a0006034b0087834b000748a300b1
:10432000f9ff32000740a00004a8be0006a8be00a6
:1043300020002000800098009200980000000600f5
:10434000889fbe008a9fbe008c9fbe000404b800f8
:104350000506b8008904460060854e000606b800d0
:104360000a054600e0854e000706b8008b054600aa
:10437000040eb800890446000a854e00e0854d0011
:10438000050eb8000a0546008b854e00060eb800e3
:104390008b0546000416b8000a0546008b854e00c2
:1043a0000516b8008b054600041eb8008b054600b4
:1043b0000800be000a01be004f06be004f05be0049
:0843c0004f04be0000000600de
:020000040000fa
:1043c80000c100008140000001c0000080410000e1
:1043d80001c000008041000000c1000081400000d1
:1043e80001c000008041000000c1000081400000c1
:1043f80000c100008140000001c0000080410000b1
:1044080001c000008041000000c1000081400000a0
:1044180000c100008140000001c000008041000090
:1044280000c100008140000001c000008041000080
:1044380001c000008041000000c100008140000070
:1044480001c000008041000000c100008140000060
:1044580000c100008140000001c000008041000050
:1044680000c100008140000001c000008041000040
:1044780001c000008041000000c100008140000030
:1044880000c100008140000001c000008041000020
:1044980001c000008041000000c100008140000010
:1044a80001c000008041000000c100008140000000
:1044b80000c100008140000001c0000080410000f0
:1044c80001c000008041000000c1000081400000e0
:1044d80000c100008140000001c0000080410000d0
:1044e80000c100008140000001c0000080410000c0
:1044f80001c000008041000000c1000081400000b0
:1045080000c100008140000001c00000804100009f
:1045180001c000008041000000c10000814000008f
:1045280001c000008041000000c10000814000007f
:1045380000c100008140000001c00000804100006f
:1045480000c100008140000001c00000804100005f
:1045580001c000008041000000c10000814000004f
:1045680001c000008041000000c10000814000003f
:1045780000c100008140000001c00000804100002f
:1045880001c000008041000000c10000814000001f
:1045980000c100008140000001c00000804100000f
:1045a80000c100008140000001c0000080410000ff
:1045b80001c000008041000000c1000081400000ef
:1045c80000c00000c1010000c303000002c20000d7
:1045d800c606000007c7000005c50000c4040000a7
:1045e800cc0c00000dcd00000fcf0000ce0e000057
:1045f8000aca0000cb0b0000c909000008c8000067
:10460800d818000019d900001bdb0000da1a0000d6
:104618001ede0000df1f0000dd1d00001cdc0000a6
:1046280014d40000d5150000d717000016d60000d6
:10463800d212000013d3000011d10000d0100000e6
:10464800f030000031f1000033f30000f2320000d6
:1046580036f60000f7370000f535000034f40000a6
:104668003cfc0000fd3d0000ff3f00003efe000056
:10467800fa3a00003bfb000039f90000f838000066
:1046880028e80000e9290000eb2b00002aea0000d6
:10469800ee2e00002fef00002ded0000ec2c0000a6
:1046a800e424000025e5000027e70000e6260000d6
:1046b80022e20000e3230000e121000020e00000e6
:1046c800a060000061a1000063a30000a2620000d6
:1046d80066a60000a7670000a565000064a40000a6
:1046e8006cac0000ad6d0000af6f00006eae000056
:1046f800aa6a00006bab000069a90000a868000066
:1047080078b80000b9790000bb7b00007aba0000d5
:10471800be7e00007fbf00007dbd0000bc7c0000a5
:10472800b474000075b5000077b70000b6760000d5
:1047380072b20000b3730000b171000070b00000e5
:1047480050900000915100009353000052920000d5
:1047580096560000579700005595000094540000a5
:104768009c5c00005d9d00005f9f00009e5e000055
:104778005a9a00009b5b0000995900005898000065
:1047880088480000498900004b8b00008a4a0000d5
:104798004e8e00008f4f00008d4d00004c8c0000a5
:1047a80044840000854500008747000046860000d5
:1047b80082420000438300004181000080400000e5
:1047c80075730000526300007642000075660000b1
:1047d80066650000725000006f730000203c000006
:1047e800204d0000425f000053450000525f00006a
:1047f80050440000555f0000534900005a4500002e
:104808005f4d000041580000002e00002e2f0000d0
:104818002e2e00002f6d00006f64000062750000ee
:10482800732f000072740000752f00006d62000085
:1048380072740000752e00006300000065530000cc
:104848006e6400005374000061740000652000006d
:104858003d3d000020530000544100005445000035
:104868005f540000585f0000494400004c450000b8
:104878000065000052630000765300007461000078
:1048880074650000203d00003d20000053540000e6
:1048980041540000455f0000525800005f49000085
:1048a800444c00004500000028200000655200002c
:1048b80063760000537400006174000065200000f6
:1048c8003d3d0000205300005441000054450000c5
:1048d8005f520000585f0000494e00004954000034
:1048e80020290000207c00007c20000028200000f7
:1048f8006552000063760000537400006174000084
:10490800652000003d3d0000205300005441000098
:10491800544500005f520000585f000052430000f9
:1049280056200000292000007c7c00002028000080
:104938002065000052630000765300007461000097
:1049480074650000203d00003d2000005354000025
:1049580041540000455f0000525800005f450000c8
:10496800525200004f5200002029000000000000b1
:10497800300000002e2e00002f2e00002e2f0000e9
:104988006d6f000064620000757300002f61000005
:1049980073630000696900002f6d00006261000008
:1049a80073630000696900002e6300000075000051
:1049b80073520000637600004275000066660000ce
:1049c80065720000506f0000732000003c2000005a
:1049d8004d4200005f530000455200005f50000048
:1049e800445500005f530000495a0000455f00002d
:1049f8004d41000058000000655300006e6400003f
:104a08005374000061740000652000003d3d000003
:104a18002053000054410000544500005f5400003a
:104a2800585f0000494400004c4500000065000044
:104a38005263000076530000746100007465000042
:104a4800203d00003d200000535400004154000068
:104a5800455f0000525800005f490000444c0000c8
:104a68004500000028200000655200006376000021
:104a78005374000061740000652000003d3d000093
:104a88002053000054410000544500005f520000cc
:104a9800585f000052430000562000002920000003
:104aa8007c7c000020280000206500005263000084
:104ab800765300007461000074650000203d00001a
:104ac8003d2000005354000041540000455f0000a1
:104ad800525800005f57000041490000545f000031
:104ae800454f000046200000290000009e060000f7
:104af800100000007606000000800000da060000c2
:104b0800400000009e06000000010000760600003c
:104b18000040000076060000000100009e0600002c
:104b280020000000c606000040000000c606000085
:104b380004000000c606000008000000da060000b5
:104b480004000000da060000080000009e060000cd
:104b5800010000009e06000000080000c6060000d4
:104b6800010000009e06000080000000760600009c
:104b780000040000760600000002000075630000d3
:104b88004e42000069740000732000003c3d0000a4
:104b980020380000002e00002e2f00002e2e0000ce
:104ba8002f6d00006f64000062750000732f000015
:104bb800667500006e630000746900006f6e000087
:104bc800732f00006d62000075740000696c0000ae
:104bd800732e0000630000004f4e00000d0a000015
:104be800004f0000464600000d0a000000000000cb
:020000040000fa
:104bf800889fbe008a9fbe00000578000204be00a0
:104c0800e50f55000f003e000a004500c13324009f
:104c1800e10578004449dd00cc41de0083017100e4
:104c28004441dd00006829008109200059ee070091
:104c3800800de9004255dd00a08c20000a054000e7
:104c4800088dbe004f05be004f04be0000000600e0
:104c5800000178006000b800e50f510004003e0034
:104c68004211dd00a08c2000020140001200be00ad
:104c780000000600e20f50002400320005003c004e
:104c88000000e00009003200e10f50004e003a0039
:104c980012003700e40f50003400320027003500be
:104ca800e50f500048003a003c003700008028001b
:104cb800c01c8800e38060008180400090ff2f00c6
:104cc8009803b60000807000c01c8800e20f5100f5
:104cd8003d003a009803a8003b00370000802800f8
:104ce800701d8800e38060008180400090ff2f00e5
:104cf800ae03b60000807000701d8800e20f5100fe
:104d080031003a00ae03a8002f00370000802800c9
:104d1800201e8800e38060008180400090ff2f0003
:104d2800c403b60000807000201e8800e20f510006
:104d380025003a00c403a80023003700008028009b
:104d4800801e8800e38060008180400090ff2f0073
:104d5800d003b60000807000801e8800e20f51006a
:104d680019003a00d003a800170037000080280077
:104d7800e01e8800e38060008180400090ff2f00e3
:104d8800dc03b60000807000e01e8800e20f5100ce
:104d98000d003a00dc03a8000b0037000080280053
:104da800401f8800e38060008180400090ff2f0052
:104db800e803b60000807000401f8800e20f510031
:104dc80001003a00e803a80000000600889fbe0022
:104dd8008a9fbe008c9fbe002a8e2000098b20006f
:104de800cb8b20000004eb00ad8620000006eb0012
:104df8006c40b90000804600028020008a007800dc
:104e0800dc1007008c2c78008c2d78000804e80052
:104e18000080200000054500e60f5400f4ff3a002a
:104e2800eb3224000005eb0008582200090020009e
:104e38000c402100120020008000eb000a007800de
:104e48008cff07000801be000a00780068ff070011
:104e58005b0078000c0878000a05e800e60f5500aa
:104e6800f4ff3a008960a9008980a90060058000e4
:104e780000c0a10000d0a00000e0a00060058800ec
:104e8800700580000000a0000010a1000020a00014
:104e9800700588009960a8009980a9008bc0a900b6
:104ea8008be0a900b00580000080a1000090a00060
:104eb80000a0a000b0058800b005800000c0a000d8
:104ec80000d0a10000e0a000b00588009bc0a800a9
:104ed8009be0a9009240a9009260a900800680008a
:104ee8000080a1000090a00000a0a000800688001b
:104ef8008006800000c0a00000d0a10000e0a00053
:104f080080068800a240a800a260a9009300a9001a
:104f18009320a900a00680000000a1006000b30053
:104f2800a0068800a00680000040a0000050a10054
:104f38000060a000a0068800a300a800a320a90084
:104f480095e0a9009600a900f006800000c0a10025
:104f580000d0a00000e0a000f00688000007800054
:104f68000000a0000010a1000020a0000007880099
:104f7800a5e0a800a600a9009640a9009660a9008f
:104f8800000780000080a1000090a00000a0a00001
:104f9800000788000007800000c0a00000d0a10022
:104fa80000e0a00000078800a640a800a660a900ad
:104fb8004f06be004f05be004f04be0000000600ad
:104fc800e20f50001800320005003c000000e0002d
:104fd80009003200e10f50002a003a000c003700a7
:104fe800e40f50001c00320015003500e50f50009a
:104ff80024003a001e003700c01c800061006000d9
:105008000009e8009803d500e30860001d00370098
:10501800701d8000610060000009e800ae03d50043
:10502800e308600017003700201e80006100600060
:105038000009e800c403d500e30860001100370048
:10504800801e8000610060000009e800d003d500e0
:10505800e30860000b003700e01e8000610060007c
:105068000009e800dc03d500e3086000050037000c
:10507800401f8000610060000009e800e803d500d7
:10508800e308600000000600e20f5000180032003c
:1050980005003c000000e00009003200e10f50006c
:1050a8002c003a000c003700e40f50001c003200be
:1050b80015003500e50f500026003a001e003700a5
:1050c8009b23ab0004003a008180fb00e11c8800b0
:1050d8000080eb0020003700b123ab0004003a0049
:1050e8008180fb00911d88000080eb001a003700ca
:1050f800c723ab0004003a008180fb00411e8800f2
:105108000080eb0014003700d323ab0004003a0002
:105118008180fb00a11e88000080eb000e00370094
:10512800df23ab0004003a008180fb00011f8800e8
:105138000080eb00080037000000eb00eb23ab0019
:1051480005003a008180fb00611f88000080eb00a9
:10515800010037000000eb0000000600889fbe0039
:105168008a9fbe008c9fbe008e1f78008006780044
:105178000006eb00e58f560019003e001104e00020
:1051880017003200010778000d8546000b33240014
:10519800610f07000004be00060037005e0f07001d
:1051a8000801500089815800e50f5100e08f59002f
:1051b8000b003e006b007d001098a300f7ff3a003b
:1051c8009e4078000d007800afff07000000e00067
:1051d800010032000c06e8005e04e000ecff3a0033
:1051e8000c0078004f0778004f06be004f05be0040
:1051f8004f04be0000000600889fbe008a1f78008a
:10520800000478008204780008007800d3ff0700c3
:1052180000057800515f2a000900e0000100320013
:10522800015f2a0008007800ccff07000a00400050
:105238004f0578004f04be0000000600e50f50003f
:1052480008003e000000400001332400610178009e
:1052580012a0a100000000006100780010a0a000ca
:1052680000000000000006000101780002f0a7001d
:105278000201ea000201ea004f11de00e20f5000cd
:105288003000320005003c000000e0000900320058
:10529800e10f500072003a0018003700e40f500088
:1052a8004c00320039003500e50f50006c003a0020
:1052b8005a003700610061004a00dd00f3bf2f008b
:1052c800d41c80008481610083017000d31c880095
:1052d8004f11dd00f0ff27009803b60000007100b1
:1052e800c01c88000000eb000100e0000100320053
:1052f8000080eb00f045880059003700610061002c
:105308004a00dd00f3bf2f00841d80008481610006
:1053180083017000831d88004f11dd00f0ff270016
:10532800ae03b60000007100701d88000000eb009d
:105338000100e000010032000080eb000046880018
:1053480047003700610061004a00dd00f3bf2f000d
:10535800341e80008481610083017000331e880040
:105368004f11dd00f0ff2700c403b60000007100f4
:10537800201e88000000eb000100e0000100320060
:105388000080eb001046880035003700610061009e
:105398004a00dd00f3bf2f00941e80008481610065
:1053a80083017000931e88004f11dd00f0ff270075
:1053b800d003b60000007100801e88000000eb00da
:1053c8000100e000010032000080eb002046880068
:1053d80023003700610061004a00dd00f3bf2f00a1
:1053e800f41e80008481610083017000f31e880030
:1053f8004f11dd00f0ff2700dc03b600000071004c
:10540800e01e88000000eb000100e000010032000f
:105418000080eb0030468800110037006100610011
:105428004a00dd00f3bf2f00541f80008481610013
:1054380083017000531f88004f11dd00f0ff270023
:10544800e803b60000007100401f88000000eb0070
:105458000100e000010032000080eb0040468800b7
:10546800000006008000eb00e50f500003003e003e
:1054780000004000e18b2000e10078000100780086
:10548800000006008080eb00e50f500005003e009c
:105498000000400001332400610078000120200052
:1054a8009080600001007800000006008080eb001a
:1054b800e50f500005003e000000400001332400c5
:1054c80061007800011020009080600001007800e1
:1054d800000006008000eb00e50f500007003e00ca
:1054e80000004000218b2000610078008080eb00e4
:1054f8000000e00001003a008000eb0001007800a5
:1055080000000600e50f500006003e00218b200039
:105518000000400000814000610078000000a10008
:1055280000097800000006008000eb00e50f50003d
:1055380007003e0000004000218b20006100780039
:105548008000eb000008a300010032008080eb001f
:105558000100780000000600e50f500009003e0039
:10556800218b20000000400000814000e10178000c
:10557800d1ff2f0001896100023324006200780006
:1055880010886000000006008000eb00e50f500066
:1055980007003e0000004000218b200061007800d9
:1055a8008000eb000018a300010032008080eb00af
:1055b8000100780000000600e50f500006003e00dc
:1055c800218b20000000400000814000610078002d
:1055d8000020a10000097800000006008000eb0010
:1055e800e50f500007003e0000004000218b20001e
:1055f800610078008000eb000028a3000100320061
:105608008080eb000100780000000600e50f5000e4
:1056180006003e00218b2000000040000081400071
:10562800610078000030a100000978000000060041
:105638008000eb00e50f500007003e00000040002e
:10564800218b2000610078008000eb000038a30067
:10565800010032008080eb000100780000000600a5
:10566800ff3ffc005268ec00000006005248ed00c5
:1056780052e8b70001003a000000fc0000000600f4
:10568800889fbe00800478000004eb00e58f54007a
:1056980006003e00f2ff07006c48b900ea0440002b
:1056a800a086200060847c00f0ff070008007800d6
:1056b8004f04be0000000600889fbe0080047800ea
:1056c8000004eb00e58f54000e003e00e4ff0700e5
:1056d8006c48b900800478006a814400a0862000e4
:1056e800e8844400e0807c008100e9001800200084
:1056f80060007900810f500001003d000004eb00bc
:10570800daff0700080078004f04be00000006001a
:10571800889fbe0080047800e58f54003b003e005f
:10572800cfff07006c48b900a8862000000044009d
:10573800c20e0700e28f54001400320005003c003e
:105748000900e00017003200e18f54002e003a00f3
:1057580011003700e48f54000600320008003500bd
:10576800e58f540028003a00ea03ab0023003a0012
:1057780025003700de03ab001c003a00220037008a
:10578800d203ab0015003a001f003700c603ab0078
:105798000e003a001c003700b003ab0007003a00c7
:1057a800190037009a03ab0017003200f01c800084
:1057b8009a03ab00fdff3a0013003700a01d8000dc
:1057c800b003ab00fdff3a000f003700501e800009
:1057d800c603ab00fdff3a000b003700b01e800087
:1057e800d203ab00fdff3a0007003700101f80000e
:1057f800de03ab00fdff3a0003003700701f800096
:10580800ea03ab00fdff3a0098ff07004f04be0013
:1058180000000600889fbe000004be00e50f54008b
:1058280009003e008eff07006c40b900a8862000e2
:1058380080004400090078006b0e0700000478001f
:105848008aff070002003700804ceb000004eb00e1
:10585800080078004f04be0000000600ae0d0700e7
:105868006242800073428000020150008381580028
:1058780010002000ea0f5100e08f590001003e009f
:105888000000eb00000006008980a9000040060027
:105898003600f800809fbe00829fbe00849fbe0035
:1058a800869fbe00f70d07009b0d07006042880029
:1058b8007142880041872000e57f2000238b20006b
:1058c8006881500064835000ea835000120037005a
:1058d800918f1200050034009e03f8005008f9006b
:1058e800208b20001000a0000d003700d01c800085
:1058f8006e00600093097000f41c800012007800ac
:1059080004587800000978009108e800960f5000c4
:1059180001003900170978009a03ab00ecff3a0040
:105928009a23a9008960a9004f03be004f02be0058
:105938004f01be004f00be003600f90000400600cf
:105948008be0a900004006003600f800809fbe00ea
:10595800829fbe00849fbe00869fbe00c90d0700bf
:105968006d0d0700604288007142880001882000a0
:10597800e57f2000438b200068815000648350003d
:10598800ea83500012003700918f1200050034009e
:10599800b403f8005008f900408b20001000a00064
:1059a8000d003700801d80006e00600093097000b4
:1059b800a41d8000120078000458780000097800bf
:1059c8009108e800960f5000010039001709780087
:1059d800b003ab00ecff3a00b023a9008bc0a900cc
:1059e8004f03be004f02be004f01be004f00be0075
:1059f8003600f900004006009260a9000040060049
:105a08003600f800809fbe00829fbe00849fbe00c3
:105a1800869fbe009b0d07003f0d0700604288006f
:105a280071428800c1882000e57f2000638b200038
:105a38006881500064835000ea83500012003700e8
:105a4800918f120005003400ca03f8005008f900cd
:105a5800608b20001000a0000d003700301e800071
:105a68006e00600093097000541e800012007800d8
:105a780004587800000978009108e800960f500053
:105a88000100390017097800c603ab00ecff3a00a3
:105a9800c623a9009240a9004f03be004f02be00d2
:105aa8004f01be004f00be003600f900004006005e
:105ab8009320a900004006003600f800809fbe0031
:105ac800829fbe00849fbe00869fbe006d0d0700aa
:105ad800110d07006042880071428800818920000a
:105ae800e57f2000838b200068815000648350008c
:105af800ea83500012003700918f1200050034002d
:105b0800d603f8005008f900808b20001000a00090
:105b18000d003700901e80006e0060009309700031
:105b2800b41e80001200780004587800000978003c
:105b38009108e800960f5000010039001709780015
:105b4800d203ab00ecff3a00d223a9009300a900ce
:105b58004f03be004f02be004f01be004f00be0003
:105b68003600f900004006009600a9000040060033
:105b78003600f800809fbe00829fbe00849fbe0052
:105b8800869fbe003f0d0700e30c070060428800b7
:105b980071428800418a2000e57f2000a38b200005
:105ba8006881500064835000ea8350001200370077
:105bb800918f120005003400e203f8005008f90044
:105bc800a08b20001000a0000d003700f01e800000
:105bd8006e00600093097000141f800012007800a6
:105be80004587800000978009108e800960f5000e2
:105bf8000100390017097800de03ab00ecff3a001a
:105c0800de23a90095e0a9004f03be004f02be00a5
:105c18004f01be004f00be003600f90000400600ec
:105c28009660a900004006003600f800809fbe007c
:105c3800829fbe00849fbe00869fbe00110d070094
:105c4800b50c07006042880071428800018b200073
:105c5800e57f2000c38b20006881500064835000da
:105c6800ea83500012003700918f120005003400bb
:105c7800ee03f8005008f900c08b20001000a000c7
:105c88000d003700501f80006e00600093097000ff
:105c9800741f80001200780004587800000978000a
:105ca8009108e800960f50000100390017097800a4
:105cb800ea03ab00ecff3a00ea23a9009640a900ea
:105cc8004f03be004f02be004f01be004f00be0092
:105cd8003600f90000400600889fbe008a1f780041
:105ce800000478008204780070082000808f50003b
:105cf80021003600208e2300e0407c00808e2300a7
:105d080060407c0080cf50001b0036006c40b9001a
:105d1800ea8e2300000545004848de008a00780026
:105d28001d0d07000000e00004003200808e2300f3
:105d3800e0407c008140e80001707c00208e230058
:105d4800e0407c00808e230060407c0080cf5000c3
:105d5800090036008a007800094078000e0d070017
:105d68000000e00004003200808e2300e0407c0048
:105d78008140e80001707c004f0578004f04be00a8
:105d8800000006000200fa00889fbe008a1f780003
:105d9800800478000004eb00f0072000808f50009a
:105da8001d003e000105d000700555000980440023
:105db8006193230061007800800f550016003100c0
:105dc800e88057000900780092fe07000000e00014
:105dd800110032000ff897000084fb004844dd00f2
:105de800098044000a05e8006193230061007800f7
:105df8008a0f500008003600e88057000900780034
:105e080084fe07000000e000030032008ff89700ce
:105e18000180fb0000044400080078004f0578006a
:105e28004f04be000080fa0000000600889fbe00f4
:105e38008a9fbe008c9fbe00299423001a8e2300df
:105e48004b9323000004eb00ec8e23008046eb000c
:105e58006c40b9000000460002102000890078005c
:105e6800c40c07000d6d7800802deb000804e800d5
:105e78000910b000e60f5400f5ff3a004f06be00c7
:105e88004f05be004f04be00000006000200fa00e5
:105e9800889fbe008a9fbe008c9fbe002a8f230069
:105ea8001b0020000004eb00640655008006eb0090
:105eb800080078006bfd07000000e00013003a00be
:105ec8006c40b900800446007ab897009a0f100019
:105ed800050032008d05780003003700aff0970009
:105ee8000800780068fc07000800780065fd0700d6
:105ef8000000e00005003a00890078006e80570035
:105f0800b90c07000000e000f4ff3a000804e800bc
:105f18006c054500e60f5400e5ff3a000b007800d9
:105f28004f06be004f05be004f04be000080fa00b9
:105f3800000006000040eb00218e23008048780016
:105f48008100e800804878008100e80080487800f7
:105f58008100e800804878008100e80080487800e7
:105f68008100e8008048780000000600889fbe0095
:105f7800499323000004eb0008007800c0fd0700e7
:105f8800802c78000804e800e60f5400faff3a0075
:105f98004f04be00000006000400fa00889fbe00ff
:105fa8008a9fbe008c9fbe00e10f2000810f500029
:105fb8000c003a006044b8001a002000080078007d
:105fc800affd07000000e000020032000850dd00cd
:105fd800890470000804e800e60f5400f7ff3a004f
:105fe8008d003700f10f2000810f500015003a0096
:105ff8008a8f23008005eb006044b8001c00200055
:106008002d0020001a00e000020032000b60dd00c5
:1060180089047000080078002efd07000000e000e9
:10602800020032000b68dd00890470000804e800f3
:106038006c0545008b85e800e60f5400f1ff3a0037
:106048007500370002f02f00000141008004eb00ca
:10605800f15f2000810f51006f003e004804de0010
:106068000804e9008880ea00c808dd008080400054
:106078006881500070072000800f510004003e0026
:10608800080078003fff07008004780062003700ae
:10609800e78f50004000320006003e00e18f5000bc
:1060a800160032000d003900e48f500059003a0004
:1060b8002300370030082000808f50003f00320056
:1060c8000080e800808f50004a00320063005000d2
:1060d800808f50004f003a003300370008007800e6
:1060e800dbfa07004e09dd004200de000000710007
:1060f800c208de008004780047003700708157002e
:10610800ee80570008007800adfb07009fbc9700a1
:10611800e6846400898444000fb89700e20f5000b9
:1061280001003a000900a0000800780041090700b2
:106138000000e000380032000930a00036003700c7
:10614800080078003afd0700090120000000e0007f
:1061580001003a008004eb00080078001ffd0700ea
:106168000000e000010032000930a00008007800bb
:1061780005fd07000000e000010032000920a00032
:1061880008007800e8fc07000000e0002200320068
:106198000910a00020003700080444006093230081
:1061a800e0047c001c0037006c44b9006a04440019
:1061b800e08e2300e0047c00170037006c40b90033
:1061c8006a004000e18e2300e1047800f00f20000f
:1061d800808f54000100360080047800c84cdd0030
:1061e800808e230060407c000080fb008084740067
:1061f80009003700080078009afc0700800478003e
:1062080009f0a7008904ea008904ea00cf4cde00ff
:10621800010037008004eb00090078004f06be003b
:106228004f05be004f04be000080fa0000000600c3
:10623800889fbe000104780002f02f000001410091
:10624800f15f2000810f510060003e00c804de00ad
:106258008904e9008980ea00c808dd0080804000e0
:1062680030082000808f50000e003e006300500070
:10627800808f500055003100e28f50002c00320012
:1062880005003e000100e00011003200e18f5000df
:106298004b003a0016003700e78f500048003e00d8
:1062a8004a00370050082000808f50003a00320022
:1062b800340039000000e800808f500043003200ad
:1062c8000000e800808f50003d003a00360037009b
:1062d8006140b8004209dd00ce01de008301710093
:1062e8004201dd000900780041fa07003700370055
:1062f800e60064008100d100120020000808a30015
:1063080001003200220020000900780059fa070035
:106318000838a30003003200090078009f0807002e
:106328002a00370009007800a50807002700370071
:106338000858a3000200320009007800f4fc0700a6
:106348000848a3000200320009007800affc0700eb
:106358000838a300020032000900780096fc070004
:106368000828a30002003200090078007afc070020
:106378000818a300150032000900780061fc070026
:10638800120037000858a3001000320009007800f6
:10639800aafb07000d003700e1006400090078003f
:1063a800b1fb070009003700208e230008f07c00ad
:1063b8008040eb00808e230001f07c000300370052
:1063c800080178000900780043fe07004f04be006a
:1063d8000000060081e0a9007d0c0700310a0700d3
:1063e8004c08070079fa070090fe0700ba0a070070
:1063f80070040700f0f12f004220b600901a8200c6
:10640800b60407000000eb00c30807008001eb009a
:10641800541a8200651a82000041eb00411a82007a
:106428000000eb0075050700090607001f060700b6
:10643800b70a070040438000f804070093fe0700ee
:106448000000e000f9ff320004fd07000000e00052
:10645800f6ff3200d90707000000e000f3ff320022
:10646800050b0700f1ff370068a8ef0013002000b4
:10647800743e2000848f500016003600010241004f
:10648800c53e2000850f520012003e008001eb003f
:106498000200e0000f003200913eb1008180400010
:1064a80042362400828040000402420022b92300c0
:1064b8000402410051017800c811de000348780049
:1064c800124098000080e800848f5000f9ff3a00dd
:1064d8008001eb000300780000000600889fbe00e2
:1064e8008a9fbe008c9fbe0080047800010478005b
:1064f800020578000306780068a8ef001b0020005a
:10650800f06f2000800f54004c003e000c00e000ab
:1065180021003a0088004500e00f2000808f5000dd
:106528000100360091fe07000a00e0001a00320060
:106538001b6020000006eb000800e900f70f500080
:1065480004003e008134240008007800220407007b
:106558000700370021f02f00888040000c007800e9
:106568008b8f500002003e00080078008afe07006a
:10657800c800de00814c7800904498008984e800c7
:106588000a05e9000804e8000a00e000eaff3a000a
:106598008005eb00290037008005eb00e10f56006d
:1065a80026003a000a00e000230032001d602000a7
:1065b8001986fb00194090008984e8004866dd00d0
:1065c8000080fb00000646000800e900f70f5000b5
:1065d80006003e00823424008c0078000800780011
:1065e80051040700800578000700370020f02f00cd
:1065f800080040008d0f500003003e008c0078001a
:10660800080078000aff0700f80f540006003a0057
:1066180020022000800f5600030036000c0078008e
:106628006f0b07003c4388000a05e90002003200ae
:106638000804e800deff37003efe07000b00780084
:106648004f06be004f05be004f04be000000060006
:106658000002be0082002000110009000202d800da
:1066680000017800e54079008181fb00720020007c
:10667800110009000202d8008000fd00120020006d
:106688000010dd0000806100000006000002be006e
:106698000200e0000a003200820020001100090018
:1066a8000202d80000017800828042006700620080
:1066b800120020000010dd00914870000a00370029
:1066c80082002000110009000202d80000017800b1
:1066d8008280420067006200120020000010dd0086
:1066e80000c0ea009148600000000600889fbe00d4
:1066f8008a9fbe008c9fbe008005780081047800c8
:106708000205780068a8ef00100020000900e000ea
:10671800e400320089004500f98f5000e1003e0096
:10672800808f51006a003a000000eb000a00e00088
:10673800dc0032000006eb000004eb002d352400dd
:106748008b00780008007800c1ff070009014600a7
:106758000082eb008082eb00cf90de000401410054
:1067680085814800f70f5100e08f590052003e0024
:1067780002600100170037001a0037001d003700bb
:106788002000370023003700260037004a00370072
:1067980049003700270037002c0037003100370048
:1067a800360037003b00370043003700420037000f
:1067b80041003700400037003f0037003e003700f7
:1067c8003d0037003c0037003b0037003a003700f7
:1067d80036003700800078000000eb00a4070700af
:1067e800350037008000780010002000a00707005f
:1067f8003100370080007800200020009c07070047
:106808002d0037008000780030002000980707002e
:106818002900370080007800400020009407070016
:1068280025003700800078005000200090070700fe
:10683800210037000000e000020032009e86a80018
:106848001d0037009e86a9001b0037000000e000ed
:106858000200320077e6a8001700370077e6a900a3
:10686800150037000000e00002003200dac6a80078
:1068780011003700dac6a9000f0037000000e00059
:10688800020032009f06a8000b0037009f06a900ef
:10689800090037000000e0000200320077c6a800b7
:1068a8000500370077c6a900030037006828ef0005
:1068b8001d007800890307000804e800080678002e
:1068c800880f55009eff3e000000eb007500370062
:1068d800500020000300e00072003a004351de003f
:1068e8000201e8008000eb000b00780055e7070084
:1068f8000000eb000a00e0006a0032000004eb0030
:106908000086eb008086eb00090040004f81de0026
:106918000c0040008d004900c40020000500200044
:10692800840f5000858f580059003e000060010018
:106938000c00370012003700180037001e0037001f
:10694800240037002a003700510037005000370074
:106958002e00370034003700390037003f00370079
:10696800450037000000eb009107070000017800a0
:106978008b0078000800780044ff070044003700c7
:10698800100020008a070700000178008b007800bb
:10699800080078003dff07003d0037002000200078
:1069a80083070700000178008b0078000800780052
:1069b80036ff070036003700300020007c0707004c
:1069c800000178008b007800080078002fff07008e
:1069d8002f003700400020007507070000017800ed
:1069e8008b0078000800780028ff0700280037008f
:1069f800500020006e070700000178008b00780027
:106a08000800780021ff070021003700f2348000d9
:106a18004411de00610161008b00780008007800f5
:106a28001aff07001a003700b23380004f11de004a
:106a38008b0078000800780014ff07001400370066
:106a4800d23680004611de00610161008b007800bb
:106a5800080078000dff07000d003700f2348000b1
:106a68004811de00610161008b00780008007800a1
:106a780006ff070006003700b23380004e11de0023
:106a8800610161008b00780008007800fffe0700b4
:106a98000804e80008007800880f55009aff3e00b7
:106aa8000000eb004f06be004f05be004f04be00bd
:106ab8000000060068a8ef00100020000000060093
:106ac8008040780000cdb30000c04000e94f50007e
:106ad80007003600f2cbb30002c1400000c0eb0053
:106ae800e54f510002003e0090ccb30000c04000ca
:106af800000006000041eb000100e0000300320046
:106b0800304141008100e900fdff3a000240ea00ff
:106b180000000600e94f500002003e000043b000ac
:106b28000a003700ea405000e5cf500002003e005e
:106b38007043b000050037008001eb00c24b2a000b
:106b4800e14b2a00001d2000a2e607000000060015
:106b5800889fbe008a9fbe00814578000204be005f
:106b680004057800d6050700a0c0b3002ae8b700de
:106b78000a02780071c0b3000801be000b4078001b
:106b8800a705070038002000e10f400005003a0083
:106b980000e22400120a0700e10f400001003a0059
:106ba8000004eb00cc050700080078004f05be0084
:106bb8004f04be0000000600c10507008000eb007e
:106bc8000080eb00ca0507002028ef00c205070077
:106bd8000000eb00620a070000000600b805070085
:106be8006000b800c2050700f8090700ba050700e9
:106bf80000000600889fbe008a9fbe0080047800bf
:106c08008105780002057800ad050700f00f200027
:106c18002c08e300050036008001eb00b24d2a0085
:106c2800e14b2a00d00920006ae607006041800095
:106c380058002000e20f50000c003600614180002f
:106c4800200a2400abff07000004e00007003a0018
:106c5800200a2400904c780060418000008de900f3
:106c6800300a2400800d78000004eb009a05070024
:106c7800080078004f05be004f04be000000060063
:106c8800889fbe008a9fbe00004578008104780076
:106c9800820578008a050700580020002008e200d5
:106ca80014003a008904e9004941880018002000ce
:106cb800384188008a4c78000b0078002628b400f8
:106cc80031418000404180008aff07003141800047
:106cd800220a240000f178008880400031418800b1
:106ce800184188008080eb000000eb008005070059
:106cf8000004eb0078050700080078004f05be0087
:106d08004f04be00000006000200fa002208e2005c
:106d1800050032008001eb0002502a00e14b2a00f6
:106d2800400e20002be607000f80e9005f050700f2
:106d380000418000e10f5000040032004900390092
:106d4800e20f500053003a00310037009c09070059
:106d58006ff89700a1c3b300814f500004003a00b8
:106d68002428ef002c28ef000000eb004c0037002f
:106d7800ed4f500004003a00200020000041880038
:106d88000000eb00460037004dff0700214180005e
:106d98000100e00003003200e18f50003f003a009c
:106da80011003700f10f200062418000810f51006f
:106db80009003e0061418000420020000200dd0021
:106dc800220a240000f178001000200020418800e9
:106dd8000000eb00320037002028ef007b09070095
:106de8000000eb002e00370061418000220a2400d9
:106df800e2c178000340700000f178008100e800eb
:106e0800614188002428ef000000eb0024003700cf
:106e18006ff897002a48e30005003a006b0907005d
:106e28002028ef0010002000cd0907001c003700c3
:106e3800a1c3b300814f500007003a002428ef0097
:106e48002c28ef0010002000004188005c09070092
:106e58000000eb00120037002028ef000000eb00d4
:106e68000f0037000000eb00a1c3b3006ff99700d3
:106e7800814f51000a003a00510907002c28ef0001
:106e88002428ef0010002000004188000000eb00db
:106e9800030037000000eb00010037000000eb00a2
:106ea8000080fa0000000600881f78002008e20031
:106eb800050032008001eb00b2512a00e14b2a00a4
:106ec800f0142000c3e5070010418000e20f5000d5
:106ed8001200320005003e000000e00040003200d1
:106ee800e10f500043003a0005003700e30f50005f
:106ef8002c003200e40f50003e003a002f0037000b
:106f0800a0c3b300e504070020002000104188005a
:106f18002428ef000004eb00370037002608e200c1
:106f28001a003200204180000000e0000400320016
:106f38000004eb00e10f50002f003a000900370071
:106f4800404180001080fb004400de00f1fe070095
:106f5800d204070010002000204188000004eb0044
:106f68002500370040418000104078006f406000e5
:106f7800e8fe0700c90407002828ec002428ef00d1
:106f88002628ed000004eb001b003700d0c0b3003a
:106f9800c204070030002000104188000004eb0004
:106fa800150037002ac8bf00bc04070040002000b5
:106fb800104188000004eb000f0037002228ef0082
:106fc8003000200066090700000478008000eb000c
:106fd8000080eb00c60407002228ef0006003700f7
:106fe8008000eb000080eb00c10407000004eb0008
:106ff800010037000004eb00080078004f04780017
:10700800000006002008ed00e10f500002003e00dd
:107018002028ef00080037002008ed00e10f50009d
:10702800050036008001eb0062532a00e14b2a007c
:10703800701a200067e50700e40807000000eb006d
:04704800000006003e
:020000040000fa
:10704c00200800000e00000080000000104300002b
:10705c0020000000800000005e080000020000001c
:10706c00800000005a0800000400000080000000ae
:10707c002e0800000a00000080000000a240000062
:10708c000001000080000000380800000a00000029
:10709c00800000006c4200004000000082000000f4
:1070ac00110070004a0400008e4903000072440075
:1070bc001000220044060000f843170000c04400f2
:1070cc0001004c0045050000ae450f0000fc4500da
:1070dc0002002e004900000000000000000000002b
:1070ec000000000000000000000000000000000094
:1070fc00000000000000000000080000200000005c
:10710c008000000060080000020000008200000007
:10711c00020000005408000006000000800000007f
:10712c006208000002000000820000000200000063
:10713c00420800000a0000008000000030430000fc
:10714c0018000000820000009a03b00003c6030080
:10715c00d203de0003ea0300a003b60003cc030055
:10716c00d803e40003f003006a0800007830000044
:10717c00800000004c0800000800000080000000a7
:10718c00e238000060060000800000006408000087
:10719c0002000000800000004843000010000000c6
:1071ac008200000001002000a10700000100000087
:1071bc00000000000000000000000000644300001c
:1071cc0008000000800000006608000002000000bb
:1071dc00820000002300000068080000020000008c
:1071ec0080000000ac4200003e0000008200000065
:1071fc002c206600756e630074696f006e3a200077
:10720c000000610073736500727469006f6e20007a
:10721c00222573002220660061696c0065643a00c7
:10722c00206669006c65200022257300222c20004a
:10723c006c696e00652025006425730025730a00b7
:10724c0000000000584300000c000000800000000b
:10725c00ea42000026000000820000006d4300009e
:10726c00006d430009000000000200006f430000a5
:10727c00006f43000e02010000000000000000003f
:10728c00000000000602020000000000ea420000bc
:10729c006c4300000600000080000000a2410000ca
:1072ac00ca00000082000000303132003334350057
:1072bc00363738003941420043444500460030001f
:1072cc0031323300343536003738390061626300af
:1072dc006465660000286e00756c6c002900000067
:1072ec00010000000000000000000a000000000087
:1072fc00000000000064000000000000000000001e
:10730c00e80300000000000000001000270000004f
:10731c000000000000a0860001000000000000003a
:10732c0040420f0000000000000080009698000012
:10733c00000000000000e100f50500000000000066
:10734c0000ca9a003b00000000000000e40b54004f
:10735c00020000000000e800764817000000000062
:10736c000010a500d4e8000000000000a0724e0040
:10737c0018090000000040007a10f3005a000000c9
:10738c000080c600a47e8d000300000000c16f00c9
:10739c00f2862300000000008a5d7800456301003e
:1073ac0000006400a7b3b600e00d000000e88900ff
:1073bc000423c7008a000000423f00006001000067
:1073cc00820000000000000000000000f03f000000
:1073dc00000000000000240040000000000000003d
:1073ec000059400000000000000040008f400000e9
:1073fc00000000000088c3004000000000000000f6
:10740c006af8400000000000008084002e4100005b
:10741c0000000000d0126300410000000000840056
:10742c00d7974100000000000065cd00cd41000061
:10743c00000020005fa002004200000000801d0040
:10744c00af1544000000000040593e0029460000e2
:10745c00000000000000f0007f00000000000000b1
:10746c0000f07f000000000000000000f07f000032
:10747c00000000000000f0007f0000000000000091
:10748c0000f07f000000000000000000f07f000012
:10749c00000000000000f0007f0000000000000071
:1074ac0000f07f000000000000000000f07f0000f2
:1074bc00000000000000f0003f00000000a0990058
:1074cc0099b93f000000000040e17a00843f0000c1
:1074dc000000e0004d6250003f00000000e0e200c0
:1074ec00361a3f000000000080b5f800e43e0000b2
:1074fc000000a000f7c6b0003e00000000a0f200a3
:10750c00d77a3e0000000000e08e7900453e000076
:10751c000000e0000b2e11003e00000000e0df0038
:10752c007cdb3d000000000000a19c00c73b00007c
:10753c00000000004c48b40039000000000020009e
:10754c006ca13700000000000000000000000000eb
:10755c00000000000000000000000000000000001f
:10756c00000000000000000000000000000000000f
:10757c0000000000000000000000000000000000ff
:10758c0000000000000000000000000000000000ef
:10759c00000000000000000000000000724300002a
:1075ac00020000008200000001000000f04a800090
:020000040000fa
:1075bc0020002000104388004a28ef004628ef00e6
:1075cc004828ef004228ef004428ef00b2a6a8009c
:1075dc0000000600010278000081eb008081eb00c6
:1075ec0002004000e0804900f70f5000e08f580087
:1075fc0035003e00006001001700370034003700f2
:10760c00330037001600370017003700180037001a
:10761c00190037001a0037002b0037002a003700fa
:10762c0029003700280037002700370026003700d4
:10763c0025003700140037001500370022003700f2
:10764c002100370014003700150037001a003700ee
:10765c001d0037001a003700400020001d003700c5
:10766c000000eb001b0037000000eb001900370096
:10767c000000eb00170037000000eb00150037008e
:10768c0010438000130037003400900011003700c5
:10769c00001020000f003700140078000d00370098
:1076ac0014009000a400900042062000030020006b
:1076bc00b7e3070007003700480407000500370050
:1076cc0030438000030037000000eb00010037005e
:1076dc006000200000000600881f7800000478007d
:1076ec00184388004a28ef000a0607003042880039
:1076fc00414288000706070010428800214288009a
:10770c000800e00002003200e40f540002003a00ce
:10771c00b2a6a90001003700b2a6a8004f04780059
:10772c0000000600889fbe0001047800f00f500096
:10773c001200320006003e008000eb00e70f500004
:10774c0030003200e80f50002d003a0007003700df
:10775c00f50f500016003200f80f50001f003200d9
:10776c00f40f500026003a0009003700080078009a
:10777c00d9ff07008000eb00220037008004eb00eb
:10778c0038019800490198008000eb001d0037007b
:10779c008801e90021002000600f2000808f51003b
:1077ac0018003e00080978008000eb001500370037
:1077bc00400620000040b8001001980021019800fc
:1077cc00820c20000241b8000068290081092000c9
:1077dc0060e307000000e900202088002100200061
:1077ec0020022000800f5400060036003843880029
:1077fc0008007800f90607008000eb000100370054
:10780c0021002000010078004f04be00000006009b
:10781c001043800000000600881f780000047800e8
:10782c00bc0507000001be0011438000e28f500030
:10783c001000320005003e000100e000090032009b
:10784c00e18f50006a003a0008003700e48f5000c6
:10785c002c00320012003900e58f500064003a0011
:10786c004f003700b2a6a90061003700b2a6a800ed
:10787c005f00370014428000254280000402510052
:10788c0085825900f05f2d0031082000800f5200d6
:10789c00818f5a0002003600b2a6a90054003700ae
:1078ac000800e000150032003042800041428000a8
:1078bc00000051008180590014032000840f5000f7
:1078cc00e08f58004a00360000022000b206b600d5
:1078dc000000e9004f00de004500dd00f1fd2f0047
:1078ec00953580008580600081007000913588009e
:1078fc0032428800434288003d003700b2a6a800ff
:10790c003b00370050428000e50f500017003e004e
:10791c0034428000454280000402510085825900a7
:10792c00e90f5200e08f5a003100360001022000ae
:10793c0094358000848060008100e900cf08de006f
:10794c00c508dd00f4fd2f009535800005026200ae
:10795c0004827000943588000000e80050428800d2
:10796c0032428800434288002100370030428000b8
:10797c00414280000000510081805900740c2000ad
:10798c00840f5000e08f580019003600b2a6a900f1
:10799c004a28ef0032428800434288001400370026
:1079ac00304280004142800000005100818059002b
:1079bc0015032000850f5000e08f58000c00360096
:1079cc0000022000b206b6000000e9004f00de0005
:1079dc004500dd00f1fd2f009435800084806000af
:1079ec008100700091358800324288004342880043
:1079fc004f04780000000600889fbe0080047800c9
:107a0c0001407800824078000403be000041e90088
:107a1c0028002000ea4f410038003e000ce8b70077
:107a2c000900e0000400320028002000e18f54001f
:107a3c0028003a0014003700e2f52300d2408800f9
:107a4c00e2f62300c240880002fc2300724088004a
:107a5c00a2f72300524088001c28ef0002012400ea
:107a6c00024088004207240012408800420c240087
:107a7c0022408800030278000601be00e9000700de
:107a8c000004780013003700025e2300d240880007
:107a9c00225f2300c24088004264230072408800a9
:107aac00e25f2300524088001c28ef00826823000c
:107abc0002408800827523001240880062802300f7
:107acc0022408800030278000601be001ffc07005c
:107adc00000478000800e00008003a009c0607004b
:107aec000000e00004003200f94088001000200083
:107afc00004388000100370038002000080078009f
:107b0c004f04be0000000600889fbe008a1f78004c
:107b1c000045780081047800280020000a04e00069
:107b2c003b003400e50107000900e00004003a00c6
:107b3c00c0262400904f150021003a002500370084
:107b4c00701382000000e0000a003200808f5400a5
:107b5c000a003200212724001000200011017800b7
:107b6c000200e00006003200828f54000e003a0042
:107b7c00030037000000eb00010037000000eb00b1
:107b8c00c200dd00c2262400810041008a48780032
:107b9c00990098000004eb00f00f50001b003a0015
:107bac0048002000190037000000e800e480400085
:107bbc00f00f5000e9ff3a00480020001300370096
:107bcc000127240010002000914f15000a003a00f4
:107bdc00010037000000eb004200dd00c12624004c
:107bec00008040000048eb000080e8000008eb003b
:107bfc000004eb00050037000000e800e4804000c2
:107c0c00f00f5000f0ff3a000004eb00b101070048
:107c1c00080078004f0578004f04be0000000600f5
:107c2c006000200001438000e18f500006003a0004
:107c3c00e14080000000eb000100e0000200320097
:107c4c00010001000000eb000000060060002000b5
:107c5c0001438000e18f500004003a00d0408000c6
:107c6c00000001006028ef000000eb00000006009f
:107c7c00014380000100e00006003a00c040800093
:107c8c000000010010002000004388000000eb0001
:107c9c000400370060002000e18f500001003a0022
:107cac000000eb00000006000200fa00600020005b
:107cbc006008e20059003a000f80e9002c0607002a
:107ccc00800078000000eb00e18f400053003a0088
:107cdc007fb89700e10f500003003200e20f500014
:107cec004d003a00150037002281200061812000f0
:107cfc005081200053408000030001008000780078
:107d0c000000eb000100e00044003a00518120002b
:107d1c00914078000cc8bf00814f50000300320026
:107d2c000000eb000104e0003c003a0020002000c1
:107d3c000a0607000000eb0038003700b040800056
:107d4c001042780041812000844878001100200006
:107d5c0081408800c1262400914078000104e00095
:107d6c0017003200814f5200080032000127240016
:107d7c0012002000914178000304e0001000320052
:107d8c00834f52000a003a00010037000001eb005b
:107d9c00c210dd008180e800c226240062817800d8
:107dac00218120000200010080408800040037007f
:107dbc000201e800e4804000f00f5100edff3a00b2
:107dcc000000eb001548e2001400320080408000f7
:107ddc000000e000090032004281200012417800ce
:107dec00b14080000274a00082487800b14080004d
:107dfc009040980020002000904088009240800025
:107e0c00b14080000cc8bf0073408000030001002b
:107e1c000000eb00010037000000eb000080fa00ce
:107e2c0000000600889fbe008a9fbe008144780037
:107e3c000205be0004047800200107000802780047
:107e4c0081c0b3000a01be0009407800f3000700ae
:107e5c0038002000e10f400010003a0030022000f2
:107e6c000100200002b02400820f5500e08f5d005d
:107e7c0005003e000a0145008b814d0000fa2700e9
:107e8c0071012000c2e107005405070038002000f2
:107e9c00e10f400001003a000004eb000d01070067
:107eac00080078004f05be004f04be00000006001d
:107ebc00020107003828ef008000eb000080eb0087
:107ecc000a0107003d05070002010700000006003b
:107edc00fa0007006000b800040107003a0507002b
:107eec00fc00070000000600889fbe008a9fbe00b1
:107efc00800478008105780002057800ef00070007
:107f0c00f00f20004008e300050036008001eb0074
:107f1c00423e2a0091402a00200a2000ace10700d2
:107f2c000042800058002000e30f50000c00360087
:107f3c0001428000200a2400710507000000e000c7
:107f4c0007003a00200a2400904c78000042800080
:107f5c00630d5000300a2400800d78000004eb0003
:107f6c00dc000700080078004f05be004f04be007f
:107f7c0000000600889fbe008a9fbe000045780066
:107f8c008104780082057800cc000700c041800095
:107f9c0058002000e10f500019003a008904e90054
:107fac00f941880018002000e84188008a4c7800cc
:107fbc000b0078003c28b400e1418000f0418000c7
:107fcc004f050700e1418000220a240000f17800ef
:107fdc0088804000e1418800e14180004800de00db
:107fec0000f1780088804000e1418800d841880089
:107ffc008080eb000000eb00bc0007000004eb00ed
:10800c00b4000700080078004f05be004f04be0006
:10801c00000006000200fa003a08e20005003200f7
:10802c008001eb0022422a0091402a00f00e200031
:10803c0067e107000f80e9009b000700c04180004a
:10804c00e10f50000a00320005003900e20f500029
:10805c0012003200e30f50001d003a0002003700fe
:10806c00d60407001a003700d404070018003700a4
:10807c004028ef0000428000210a24006ff997008d
:10808c00827078000000e800004288002000200088
:10809c00c0418800c90407000d003700f00f200014
:1080ac004008e30007003e0000428000210a240043
:1080bc006ff99700827078000000e8000042880099
:1080cc000200370030002000c0418800bb040700cc
:1080dc000000eb000080fa0000000600881f78000a
:1080ec00c0418000e10f5000050032008001eb0020
:1080fc00d2432a0091402a00a012200034e107004c
:10810c00d04180000000e000040032000004eb00cd
:10811c00e10f500016003a00050037008000eb001c
:10812c000080eb00710007000004eb00100037002a
:10813c003c08e20007003200f0418000104078005b
:10814c00550007003e28ec003c28ed000004eb0035
:10815c0007003700300020000005070000047800fd
:10816c008000eb000080eb00600007003a28ef0075
:10817c00080078004f04780000000600881f780083
:10818c00c0418000e20f500007003200e30f5000a6
:10819c00170032000000e00007003a00ef0407006f
:1081ac00000478001700370010002000eb040700d3
:1081bc0000047800130037003808e2000e0032008b
:1081cc00c0418000e20f50000d003200c041800021
:1081dc000004eb00e30f50000a0032008001eb00ba
:1081ec0082452a0091402a0040162000f8e0070042
:1081fc000004eb00030037000004eb000100370023
:10820c000004eb007004070010002000c04188003f
:10821c00080078004f047800000006001020800051
:10822c00002080008920a9008f40a9008940a90066
:10823c0010182000a01f880000012300b01f880028
:10824c0000022000e01f88008000200040208800f1
:10825c00001028005020880090002000202088006a
:10826c00200680000030b30000a0a100200688008a
:10827c00600580000080a1000090a00000a0a1007b
:10828c00600588009f40a9009940a900f5e3a8006b
:10829c000080eb00000006000000fb0000208800be
:1082ac000080eb0000000600218320009140780044
:1082bc00014878000080eb0000000600f0f92f0068
:1082cc004200b6000070a000100288003668ec0076
:1082dc00000006003648ed0036e8b70002003a0010
:1082ec00f0f12f004220b60000000600889fbe006f
:1082fc008004780001047800f0ff07000900e0001a
:10830c001d0032003408e200030032000108200096
:10831c00fce3ab000400320001022000fca3ab0024
:10832c00060032000d00370000000000e21f800044
:10833c0002806000fcff3200f7ff37000020800055
:10834c0000417800e31f800003806000fbff3200d7
:10835c00824078002083200001487800fcc3a900eb
:10836c00f5e3a90010182000a01f88008f40a90079
:10837c009f40a800010037009f40a900a841880039
:10838c000800e00006003200f5e3a90010122000fe
:10839c00a01f88008940a8009940a800020037005f
:1083ac009940a9009f06a900f5e3a800c9ff0700a2
:1083bc004f04be00000006000000eb003408e20091
:1083cc000b003a00d3020700724180008341800009
:1083dc00020150008381580011002000ea0f510067
:1083ec00e08f590001003e008000eb000100780096
:1083fc00000006003600f800809fbe00829fbe0081
:10840c00849fbe00869fbe001d0307008940a90003
:10841c009f06a8003408e20008003200fc23ab00e1
:10842c0006003a0010408000000001003408e20011
:10843c0002003200fc23ab00faff32009f06a900b9
:10844c004f03be004f02be004f01be004f00be00e6
:10845c003600f900004006003600f800809fbe0090
:10846c00829fbe00849fbe00869fbe00881f78003e
:10847c00030307008f40a90077c6a800a5020700d8
:10848c007041880081418800fcc3ab0004003a00b5
:10849c0008022000fca3ab000e00320014003700d1
:1084ac00fca3ab0009003a0002022000002080006f
:1084bc0080407800e31f800003006100fbff320066
:1084cc00014178002083200002487800fcc3a900f9
:1084dc00070037000020800032e8b7000040800021
:1084ec0000000100e31f800003006400f9ff32006c
:1084fc0077c6a9004f0478004f03be004f02be00a0
:10850c004f01be004f00be003600f90000400600cf
:10851c006626ef007a26ef008e26ef00a226ef00eb
:10852c00b626ef00ca26ef00de26ef00f226ef009b
:10853c000627ef005e26ef0000002900303488008b
:10854c0041242000d1348800ae26ef000101200028
:10855c0011368800ea26ef00fe26ef000107210005
:10856c009133880001282000b1368800810020005a
:10857c00b13388006226ef00503488009e26ef004d
:10858c00b226ef00c626ef00da26ef00ee26ef004b
:10859c000227ef0000000600e50f500006003e0029
:1085ac004200dd00a2572a00e20078000080e800bb
:1085bc00620078009108700000000600e50f500082
:1085cc0007003e004200dd00a2572a00e2007800be
:1085dc000080e800620078000080ea0091086000ea
:1085ec0000000600e50f500010003e000100e00006
:1085fc00070032004200dd00a2572a00e20078009a
:10860c000080e800620078009108700007003700d5
:10861c004200dd00a2572a00e20078000080e8004a
:10862c00620078000080ea009108600000000600fb
:10863c00800078000000eb00e58f50000a003e003f
:10864c00c208dd00a0572a00608178008180e80014
:10865c00608078001200600000f0a7000000ea00c3
:10866c000000ea004f00de0000000600889fbe00fc
:10867c008a1f780080047800e58f540022003e00a9
:10868c00b2c6a8000100e0000e003200c348dd00b5
:10869c0020592a00608578008180e8006084780089
:1086ac001a0d7400400020001e0207000884ea0026
:1086bc001a0d6400100020000900dd006428b700ca
:1086cc0010003700c348dd006481400020592a00a7
:1086dc0060057900e6804000608478001a0d740013
:1086ec00400020000f0207000884ea001a0d640005
:1086fc00100020008904dd008984ea0040862000f7
:10870c0010886400b2c6a9004f0578004f04be0063
:10871c0000000600889fbe0080047800b2c6a80046
:10872c0028592a00880078000000eb0000c9de0000
:10873c000208a3000400320011017800910190009e
:10874c00128971000300370021019000b1019000e3
:10875c00128971000000e800e8804000e60f50002c
:10876c00f2ff3a0040002000ee010700225c2a00d4
:10877c0018007800980090008180ea001088600052
:10878c0028009000b80090008180ea0010886000fa
:10879c0068044400820f5400f5ff3a00b2c6a900e9
:1087ac00294388004f04be000000060080007800ba
:1087bc000000eb00e58f500007003e001000200089
:1087cc000100dd006408b60000f0a7000000ea001c
:1087dc000000ea004f00de0000000600204380008d
:1087ec00000006003200200053002000918f110081
:1087fc000f003a00104190004811dd00a04090009d
:10880c008180fb00828070008100e80063004000e2
:10881c0013002000030178002ff707000001eb0084
:10882c000000e00002003200460207000001780060
:10883c000200780000000600881f78000104780010
:10884c003300200051002000988f10001f003600cc
:10885c0090409000a0439000b0419000c819dd00fa
:10886c00404190000281fb000301710050439000d5
:10887c008202e9003300200074072000848f52002c
:10888c0012003e0002424100864f52000f003a0097
:10889c00c808dd008783fb00818073008100e8003d
:1088ac0066004000130020000bf707000000e000fa
:1088bc000300320023020700800178000300370018
:1088cc0050002000000c78008001eb0003007800c1
:1088dc004f04780000000600889fbe000104780059
:1088ec003200200051002000988f10001e003a002a
:1088fc0080017800d3407800a04390004042900063
:10890c008484fb000903e900c5072000850f530090
:10891c0015003e00000ceb0002487800180ce80033
:10892c000300780004584200180ce800c808dd0069
:10893c008783fb00818073008100e8008001eb00dd
:10894c0009017800e4f607000000e00003003200a3
:10895c00fc01070000017800030037008984440003
:10896c00188c44000001eb00020078004f04be009c
:10897c0000000600889fbe008a9fbe008c9fbe0030
:10898c000004be000000eb0091002000998f100045
:10899c003a003600080578005a467800a846900040
:1089ac00b8459000c85ddd00484090000080fb0099
:1089bc008b057000d843900068439000784190007c
:1089cc00084a9000984a90008b01e9003000200082
:1089dc00c1072000818f510028003e004811dd00a6
:1089ec000482fb000201720024003200e38050007c
:1089fc00810f510021003e00820041008582fb0066
:108a0c00858f50001d003a00c838dd000683fb003e
:108a1c00810073008100e8006a004400130020000c
:108a2c00adf607000000e00013003a00800ceb00ec
:108a3c0070c1b300004c7800990ce8000a00780073
:108a4c000bd84500990ce800c860dd008d86fb0052
:108a5c00818076008100e8008001eb000b0178003a
:108a6c009df607000000e00003003a008b854500ee
:108a7c00998c450001003700b20107004f06be007b
:108a8c004f05be004f04be0000000600889fbe00cc
:108a9c00010478003300200051002000988f100052
:108aac0028003a0000027800d4407800a0439000df
:108abc00b0419000c819dd00404190000281fb00dc
:108acc00030171000203e90033002000e57c200063
:108adc00850f53001b003e00000ceb0013c0b300cd
:108aec0003487800180ce8006700610003003200ae
:108afc00c314de008944e80001003700c314de0013
:108b0c000400780009587800180ce800c808dd004b
:108b1c008783fb00818073008100e8008001eb00fb
:108b2c00f1f607000000e0000300320085010700a9
:108b3c0080017800030037008984fb00188c440006
:108b4c008001eb00030078004f04be00000006001b
:108b5c000200fa003200200053002000918f110017
:108b6c001f003a009040900020429000c0419000bd
:108b7c000304e0001a003a00304090008041e90004
:108b8c00e3cf4100160036000041eb00f2ff9f00de
:108b9c00e14f400003003a0010c0b300e0ff9f001b
:108bac00020037000040eb00e0ff9f00c808dd002a
:108bbc000482fb00810072008100e8001300200099
:108bcc00030178000f80e900c7f607000001eb00f5
:108bdc000000e000020032005a010700000178009a
:108bec00020078000080fa0000000600889fbe009a
:108bfc00010478003300200051002000988f1000f1
:108c0c002400360090449000a0409000b0419000a9
:108c1c00c819dd00404190000281fb000301710086
:108c2c0050439000e701610003003200c313de00e3
:108c3c008743e80001003700c313de008202e9001d
:108c4c0033002000f47a2000848f520011003e0083
:108c5c0086cf53000f003a00c84cdd008180fb002a
:108c6c00898070008100e80066004000130020003d
:108c7c009df607000000e000030032003101070000
:108c8c00800178000300370050002000000c7800b1
:108c9c008001eb00030078004f04be0000000600ca
:108cac000ca1a90000fc2f00a23d800082006000f6
:108cbc007101b300a13d8800533f80008300600028
:108ccc003100b300513f8800b23d8000820060004b
:108cdc00a100b300b13d8800f10f2c00223f8000b1
:108cec00828160000250200003017100223f880045
:108cfc00923d80008281600002a02100030171007e
:108d0c00923d8800323f8000828160000230210059
:108d1c0003017100323f8800333e80000301600084
:108d2c000220a000323e8800b23e800082816000aa
:108d3c000250210003017100b23e8800c23d800048
:108d4c00828160000220210003017100c23d880075
:108d5c00333f8000030160000230a000323f8800e6
:108d6c00c33d800003016000c201b300c23d880016
:108d7c00023f8000828060000270200001017100bf
:108d8c00023f8800ba07b6006000b300d03d8800ef
:108d9c00d2fb2f0003088000030161000260a000d9
:108dac007105200060042000031020008049780029
:108dbc008149780082497800000000007801a80001
:108dcc007861a9007881a8008201a8008221a800fe
:108ddc0078a1a90078c1a9007c61a9007ea1a90095
:108dec0086c1a90086e1a90078e1a8007c21a80031
:108dfc007c41a8007961a9007981a90079a1a90019
:108e0c0079c1a90079e1a8007a01a8007a21a8000b
:108e1c007a41a8007a61a8007a81a8007aa1a800fa
:108e2c007b01a8007b21a8007b41a8007b61a800e6
:108e3c007b81a8007ba1a8007d01a8007cc1a800b3
:108e4c001381a8007d41a8007ce1a8007ce1a8006a
:108e5c007e01a8007e01a8007e21a8007e41a8000a
:108e6c007e61a8007c21a8007e21a8008001a800ba
:108e7c008021a8008041a8008061a8008081a80002
:108e8c0080a1a80080c1a80082c1a8008481a8008c
:108e9c0084a1a8008601a8008641a8008661a800cc
:108eac008681a80086a1a80000000600b4428000bc
:108ebc00c5428000a0428000040150008001eb00fc
:108ecc000200420083804a00b0428800c142880000
:108edc000000060000012000000d8800300d23006a
:108eec00e00c88009621ef005005800000c0a00027
:108efc0000d0a10000e0a0005005880088e0a90087
:108f0c0098e0a800a1e1a80000000600e7ff070018
:108f1c0000000600e5ff0700b0428000c14280005f
:108f2c0000000600889fbe0000047800f9ff0700cf
:108f3c0000044400e0844800f6ff0700800f540052
:108f4c00818f5c00fcff3e004f04be000000060059
:108f5c00713e2000810f5000060036006900400071
:108f6c00a2002000110009000280d800edff0700cc
:108f7c001a0037000000e000180032000102200047
:108f8c00110d88009a21ef008000eb00820920006f
:108f9c000281b900046829000400b8008100410076
:108fac0002a02f00030020006add07000000e9008a
:108fbc00f00c88009900a9008900a900a3e1a80081
:108fcc008900ab0005003a000110200000000000f1
:108fdc004204800002806000fcff320000000600aa
:108fec0071382100810f5000060036004038b00067
:108ffc00823e2000110009000280d800d4ff070037
:10900c0016003700f40f500014003600a221ef00b8
:10901c009a21ef0074005000811a26000100b8005c
:10902c00429c2000030020004add07000000e900fc
:10903c00f00c88009900a9008900a900a3e1a80000
:10904c008900ab0005003a00011020000000000070
:10905c004204800002806000fcff32000000060029
:10906c007666a8005428ec0088e0a9007666a90072
:10907c00004006000361a800dac6a8000000060044
:10908c000361a900dac6a90000000600e84f5100f0
:10909c00050036008001eb00225c2a00f15c2a00fe
:1090ac00800320004add0700430bde00e7826000ee
:1090bc008381fb000281fb00110020000209dd000e
:1090cc000201e900060240009483fb000103430007
:1090dc00060040009080fb00c808dd008180730012
:1090ec000511dd000281ea0082806000851add0036
:1090fc0081807200014a7800c808de0001487800bf
:10910c0000000600c309de0060c279000482fb0087
:10911c0003004000104090004800dd000000720089
:10912c00c319dd00838050000100de000281fb00ca
:10913c00110020000209dd000201e90002006000bc
:10914c00000006008000780020002000e18f500015
:10915c00060032000000eb00040039006000200023
:10916c00e78f500001003200400020000000060094
:10917c0001087800110098002100980082804000be
:10918c0031009800420098008000eb0051009800dc
:10919c0000000600410190000201e900510290001c
:1091ac008001eb00820f52000c003d001101900079
:1091bc000059780092009800510090000000e800df
:1091cc00d00098003100900013002000800f510057
:1091dc00020039001100780090009800030078001c
:1091ec00000006002101900091019000830f5100b6
:1091fc0004003a000048eb000000eb00d00098009f
:10920c000c00370032487800a20098005100900002
:10921c000000e900d0009800b1019000100020007f
:10922c00830f51000300390011007800a000980052
:10923c00100020000000060090007800110098003b
:10924c00210098008000eb005100980000000600ff
:10925c00889fbe00010478003300200051002000dc
:10926c00988f100027003a0000027800d440780054
:10927c00a0439000b0419000c819dd00404190001f
:10928c000281fb00030171000203e900330020009e
:10929c00e57c2000850f53001a003e00000ceb000b
:1092ac0023c0b30003487800180ce8006700610085
:1092bc0003003200c314de008944e80001003700cb
:1092cc00c314de000400780009587800180ce8007c
:1092dc00c808dd008783fb00818073008100e800f3
:1092ec00f3f507000000e0000300320095ff0700d3
:1092fc0080017800030037008984fb00188c44003f
:10930c008001eb00030078004f04be000000060053
:10931c00889fbe000104780032002000510020001c
:10932c00988f100022003a0080017800d34078001a
:10933c0020439000b0449000c84cdd0040419000a8
:10934c000281fb00890471008902e90032002000cf
:10935c00b4072000848f520015003e00000ceb0077
:10936c0042c0b30002487800180ce80003007800f3
:10937c0009d84400180ce800c808dd000683fb007f
:10938c00810073008100e8000901780035f40700c2
:10939c000000e000030032006aff070000017800c3
:1093ac000300370089844400188c44000001eb0052
:1093bc00020078004f04be00000006009021ef0070
:1093cc0095e1a80000000600bcfb070095e1a90090
:1093dc008860a900bffb070000000600889fbe0044
:1093ec00000478000000eb00f30f54000d00360071
:1093fc00f5ff0700401f200000c4b900980c88003e
:10940c009421ef004005800000c0a10000d0a00016
:10941c0000e0a100400588009860a8008860a900c1
:10942c000080eb004f04be00000006003600f80080
:10943c00809fbe00829fbe00849fbe00869fbe00a0
:10944c008860a90020408000000001004f03be008e
:10945c004f02be004f01be004f00be003600f900a7
:10946c0000400600881f7800020278000384e800a0
:10947c0045002000ff0f540013003e000231240071
:10948c00004978000040eb000100e00001003200d0
:10949c0000c0eb001131240080487800200020002f
:1094ac00f04288008002eb000300e000060032006e
:1094bc0003017800840078002031240059dc070077
:1094cc00f84288008002eb00050078004f04780019
:1094dc0000000600889fbe0081047800f8428000de
:1094ec000000e80008017800013124004ddc070081
:1094fc00880ce8000000eb004f04be0000000600e2
:10950c000100e0000c00320080c1eb000342780047
:10951c00461e2a00452e2a0030c169000281fb003c
:10952c00e641790083416a00654279008100e900d7
:10953c00f9ff3a000200370080c1eb0003427800cb
:10954c004820dd008381fb000080710000000600d4
:10955c005a28ef000080eb00000006008000780025
:10956c000080eb00d0428800e14288000000060039
:10957c00800078000000eb005a08e2000400320082
:10958c00e0428000800878005a28ef000080eb0051
:10959c0000000600710520000001eb0060042000b3
:1095ac0003102000804978008149780082497800b6
:1095bc0000102400100888000621ef006821ef003d
:1095cc006a21ef006c21ef0000000600f1ff07009c
:0495dc000000060085
:020000040000fa
:0495e0000000000087
:020000040000fa
:020000040002f8
:04af0000ffff00004f
:020000040000fa
:020000040002f8
:04af3000faffff0025
:020000040000fa
:020000040002f8
:04af38009effff0079
:020000040000fa
:020000040002f8
:04af40009fffff0070
:020000040000fa
:020000040002f8
:04af48007fffff0088
:020000040000fa
:020000040002f8
:04af5000dfffff0020
:020000040000fa
:020000040002f8
:04af58003fffff00b8
:020000040000fa
:020000040002f8
:04af6000ffffff00f0
:020000040000fa
:020000040100f9
:04300000ffffff00cf
:00000001FF
